:10000000F01F0010CD4A0000C94A0000C94A000094
:10001000C94A0000C94A0000C94A000000000000A7
:10002000000000000000000000000000C94A0000BD
:10003000C94A000000000000C94A0000251C000059
:10004000AD1B0000AD1B0000AD1B0000AD1B000090
:10005000AD1B0000AD1B0000AD1B0000AD1B000080
:10006000AD1B0000AD1B0000AD1B0000AD1B000070
:10007000AD1B0000C54A0000C54A0000F51D000088
:10008000E91C0000011D0000F52000004D210000CA
:10009000C54A000055220000C54A0000C54A0000BC
:1000A000C54A0000C54A0000C54A0000C54A000014
:1000B000C54A0000C54A0000C54A0000C54A000004
:1000C00070B5041C00200D1C00F094FF002801D026
:1000D00002F09EFC00262E60201C2660291C00F0E9
:1000E000B7FF301C00F086FFB04207D002F090FC52
:1000F0002E60201C2660291C00F0AAFF70BD08B5E8
:1001000001F0C2FD08BD08B500230B60036000F0DC
:100110009FFF08BD10B502F043FC0D4B002019688D
:1001200002F060F8002002F04BF8002001F0EEFF32
:10013000084B01241C60084B201C198801F01EFE8E
:10014000201C01F009FE201C01F0E6FD10BDC04698
:1001500064050010680300106C05001008B50A2043
:10016000002101F019FDFFF7D5FF08BD08B50020FB
:1001700001F0DCFF012001F0DFFD02F017FC08BDFB
:1001800038B50D1C041CFFF7C5FF054B0122291CC7
:100190005A62201C03F0BCFFFFF7E8FF38BDC046E1
:1001A000400D001010B5041CFFF7B4FF201C03F035
:1001B00037FF041CFFF7DAFF201C10BD08B5002034
:1001C000FFF7F0FF08BD000008B5021C0249034814
:1001D00002F06AFA08BDC046044D0000FC4C000065
:1001E00013B500F06BFD154800210322144B00F0FD
:1001F00059FE00F06DFDFFF7E1FF1248FFF7E4FF45
:10020000002402F011F9002803D001F0E7FA0024DD
:1002100009E00A2001F038FD684601A9FFF750FF08
:10022000009B002B03D1084B01349C42E9DDFFF712
:10023000C5FF064802F038FA13BDC0460D4D000058
:10024000080000101C4D00006F170000224D000038
:100250007047000073B5194B041C1949186804F065
:10026000B7FC18490090184A184B201C02F027FAD6
:1002700000F0CCFF002812D000F0E4FFFA21890042
:10028000051C04F0A5FC061C201C02F065FA104BAE
:10029000201873430F49EB18321C02F010FA201C8F
:1002A00002F05AFA0C4B20181B68002B01D00B4AA5
:1002B00000E00B4A0B4902F002FA73BD680500101A
:1002C00040420F00304D0000044D00003D4D000045
:1002D00018FCFFFF414D00003C0200106E5600006C
:1002E0002D4D00004C4D000070B5051C0C1C161C5B
:1002F00000F0E4FC291C201C0022064B00F0D2FD7B
:10030000301C01210922044B00F0CCFD00F0E0FC80
:1003100070BDC046080000101400001038B50D1C58
:10032000041C00F096FC2A1C0120211CFFF7DCFFB6
:10033000034B00225A60034A943212689A6038BD17
:10034000400D0010A405001000B5084B89B01A78C4
:10035000074B68461B78074902F0B1F9694601204E
:10036000054AFFF7C1FF09B000BDC04630020010CA
:1003700010000010534D0000614D000073B5264B76
:1003800000241D78254B1E78FFF7DEFFFFF716FFD0
:10039000684601A9FFF794FE009B002B26D0182B7E
:1003A00031D004DC142B0ED0152B1AD106E0352BDE
:1003B0000BD0842B2DD0342B13D10CE0164B1A7894
:1003C0003E2A0ED805E0144B06E0144B1A78062A94
:1003D00007D8013204E0114B1A78002A01D0013A03
:1003E0001A7000F057FCFFF7AFFF0024009B002BB2
:1003F00002D0C82001F048FC04200321013401F0A0
:10040000CBFB1D2CC4DD044B1D70044B1E7000F093
:1004100041FCFFF7D3FE73BD300200101000001046
:1004200010B590B0041C6846FFF714FF69466A4691
:10043000201CFFF759FF10B010BD000010B58CB0A4
:100440002D22002800D02B2208AC201C0C4902F0E1
:1004500036F9684602F06CFB0120211C6A46FFF762
:1004600043FF0320002101F097FB0220FFF79AFED3
:100470000028EED00A20002101F08EFB0CB010BD48
:10048000A14D0000F7B502F0E9FA18200021FFF7AE
:1004900077FE0024674EFFF769FE674B674D002229
:1004A0005A629835201C02F0FAFA002C02D0002083
:1004B000012101E00620032101F06EFB201C02F067
:1004C000E9FA01A9071C684603D0FFF71CFE0127C3
:1004D00026E0FFF718FE009B002B21D1002CE1D174
:1004E0002B68002B0DD0564B00941A6811321A60FD
:1004F00004E003F03FFD009B01330093009B102BB1
:10050000F7DD504BF618CDD518200021FFF738FE47
:100510004A4B94331C6863425C4100F083FBC1E7A3
:10052000002C0CD0002F02D1009B182BB3D100F06F
:10053000D7FB4548FFF748FE404B0122DA6600F042
:1005400093FE02F0E5F9009B182B5BD1019E00247D
:10055000F0B200F0C3FC384B012501945D6217280E
:1005600038D00AD813281AD002D8112847D10FE062
:1005700015281CD0162842D121E0262822D002D8E6
:1005800019283CD10EE044282CD0452837D12EE044
:100590002E4B1B68002B35D002F0AEFB32E0FFF78C
:1005A0001FFE2FE02A4B1868281A00F08BFF01204D
:1005B000FFF736FFFFF702FEFFF7D0FD22E0FFF75F
:1005C000DDFE1FE0234B05221C70234B1A7000F048
:1005D00061FB17E0214B1A6801321A60032A11D11E
:1005E0001C600FE01E4802F02BFB201C04E0E12001
:1005F000000102F025FB281CFFF720FF02E000228B
:1006000001965A62FFF786FD0098019903F080FD7C
:10061000094B5B6A002B01D0FFF7D0FD074B9433E9
:100620001B68002B03D100F0FDFA012432E704F02F
:10063000E7F92EE720BF0200400D0010A4050010CE
:100640007C0300100CFEFFFFAA4D00003C020010CE
:1006500020000010300200101000001008020010EE
:10066000F0F1FFFF73B5314C02F0BCF800F082FCF2
:100670002F48002101F046F900212E4801F042F9EF
:1006800000F054FD00F0FAFE23680725AB43236019
:1006900023680126334300202360021C0B2101F054
:1006A000BFF8201C244C102101F02CF923680022F3
:1006B000AB4323602368301C2360042101F0B0F8B1
:1006C000201C002101F01EF901F094F89620000290
:1006D00001F0FEFD194D2824201CFFF7A1FEFA2091
:1006E00001F0D2FA02F086F9282C02D1281C01F080
:1006F000DBFF01F099FE002802D0FFF771FD02E058
:10070000043C032CE8DC02F045FC03F053FB1E2301
:1007100000930F2301930A480A490B4A0B4B03F03D
:100720005BFB0B4803F08AFBFFF7ACFE7440044010
:10073000984004409C40044094400440B44D000064
:10074000814A0000C10000001D0300007C0300106E
:1007500068030010F7B5031C00383BD01A78303A14
:10076000504242419B181A78782A03D1013310264F
:10077000012501E00A2600251A7800242D2A01D13E
:1007800001330124002201951CE0071C303FFDB21B
:10079000092D02D87243D21913E0019D002D0BD010
:1007A000202528436625854206D36025854203D24D
:1007B00012015738024304E0074801F075FF00209A
:1007C00008E0013318780028DFD1002C00D0524215
:1007D0000A600120FEBDC046BE4D000000B500E02D
:1007E00001300378202BFBD000BD00B5031C303B4B
:1007F000DAB2092A01D8181C08E020231843031C88
:10080000613B5738052B01D90120404200BD70B52E
:100810000E1CFFF7E3FF0025041C06E0FFF7E5FFD1
:10082000002805DB2D010543013420780028F5D18F
:100830003560201C70BD000008B500F003FD011CF0
:10084000014801F031FF08BDCC4D000000B589B072
:10085000684602F06DF96946024801F025FF09B0CB
:1008600000BDC046084E0000F7B50E1C01A9171CBC
:10087000FFF770FF002814D0019D0B49281C04F0DD
:10088000FDF90C1C081C642104F0F8F9201C3170DF
:10089000642104F09DF904493870281C04F098F98B
:1008A00001E001204042FEBD1027000037B50C1CBE
:1008B00048686A46694607310632FFF7D5FF01AD41
:1008C00069466A4628800132A0680231FFF7CCFFF2
:1008D0006B4618702A88044B9A4203D9281C694633
:1008E00002F095F937BDC0466B07000007B54868B0
:1008F00001A9FFF72FFF01983C23584302F0A0F90C
:1009000007BD000000B5C300181A064BC018072326
:10091000013BC25C002A03D1002BF9D1012000E089
:10092000002000BD400600107FB5194801F0BCFE54
:1009300000250326354219D1281CFFF7E3FF0028C4
:1009400010D0681CFFF7DEFF00280BD0A81CFFF7B3
:10095000D9FF002806D0E81CFFF7D4FF002801D0FB
:1009600004350FE00B48291C01F09EFE291C684647
:1009700002F034FB684601F04FFF074801F094FE97
:100980006C1C251CFF2DD5DD01F054FF7FBDC0463A
:10099000044D0000D84D00008494000070B50E1C7A
:1009A000FFF71CFF0D25041C2078FFF71EFF002811
:1009B00007DB01347055013DF6D2201CFFF70EFF16
:1009C00000E0002070BD000030B5434C87B02368C4
:1009D0000868002B06D1414801F066FE03F0EAF9F1
:1009E000012351E0012B0CD13D49082201F0C7FE43
:1009F000002802D12368013346E03A4801F054FE52
:100A00005EE00378412B1BD1374C0230211CFFF7ED
:100A1000C5FF002854D00378422B51D1211C02304D
:100A20000E31FFF7BBFF00284AD00378432B47D194
:100A3000211C02301C31FFF7B1FF002849D13FE0F3
:100A40004D2B23D1294D0230291CFFF7A7FF002889
:100A500036D003784E2B33D1291C02300E31FFF7EC
:100A60009DFF00282CD00378472B29D1023005A9FF
:100A7000FFF7CDFE059B002B22DB2A3D6B651C4852
:100A80001C4901F011FE0023236022E005A9FFF7B5
:100A9000BEFE0378041C202B01D0002B10D10025B2
:100AA000201C01A9FFF77AFF0599041C691801A809
:100AB00002F0A8FA002C03D00135042DF0D108E093
:100AC00003F078F90A480C4901F0EEFD024B0022D0
:100AD0001A6007B030BDC04640030010E14D000071
:100AE000044D0000F74D0000A4050010CE050010D5
:100AF000034E00007A4D00000D4E000037B54C68E3
:100B000024E0201CFFF76AFE01A9FFF780FE019B8D
:100B1000041C002B1DD0D8B2FF2B09DD00F0FAF920
:100B2000051C01980012C0B200F0F4F9019003E036
:100B300000F0F0F9002501900198002802D0291C4E
:100B4000FFF71EFB23785A1E9341E4182378002BED
:100B5000D7D137BD08B5064A012113784B40137031
:100B600001D0044900E00449044801F09DFD08BD9E
:100B700058040010B14D0000144E0000184E000043
:100B800070B5051C01200821021C00F097FE072407
:100B9000012601200821002200F090FE2A1C22419B
:100BA00032400020022100F089FE01200821021CB1
:100BB00000F084FE013CECD270BD10B50021041C95
:100BC0000A1C022000F07AFE201CFFF7D9FF10BD9E
:100BD000F7B5012300930023019372B66C46061CFF
:100BE00002AF01CC50235B421843C0B2FFF7E5FFD0
:100BF0000020FFF7E2FF1020FFF7DFFFE020FFF704
:100C0000DCFF002502200021012200F057FE705D6C
:100C10000135FFF7B5FF842DF4D18436BC42E0D115
:100C200062B6F7BD08B5AC20FFF7C7FFAE20FFF7EF
:100C3000C4FFA520FFF7C1FF08BD38B50D1C041C7B
:100C4000012200F0EDFD291C201C012200F036FEDF
:100C500038BD08B5AF20FFF7B0FFA420FFF7ADFF08
:100C600008BD08B5AE20FFF7A8FF08BD10B5041CED
:100C7000F820FFF7A2FF201CFFF79FFF10BD10B563
:100C8000041C8120FFF799FF3F202040FFF795FFCC
:100C900010BD000008B5074B20201B781843FFF754
:100CA0008CFF0A2000F0F0FF034B1878FFF7E7FFF6
:100CB00008BDC046100000103002001008B58422A4
:100CC00002480021520001F027FD08BD5904001020
:100CD00008B50248FFF77CFF08BDC0465904001064
:100CE00008B501200821FFF7A8FF00200221FFF727
:100CF000A4FF02200021FFF7A0FF02200621FFF73A
:100D00009CFF0320011CFFF798FF0320011C002219
:100D100000F0D4FD02200621002200F0CFFD0621C4
:100D20000122022000F0CAFDFFF7C8FFFFF7D0FF45
:100D3000A220FFF742FFA020FFF73FFFC020FFF7F0
:100D40003CFF0020FFF792FF0A2000F09DFF4020AB
:100D5000FFF733FF2C20FFF730FF322000F094FF25
:100D60002E20FFF72AFF322000F08EFF2F20FFF702
:100D700024FF0A2000F088FFFFF78CFFAF20FFF769
:100D80001CFFA420FFF719FF08BD000000B50F29C4
:100D90000ED883280CD8CB08842253430722C018CE
:100DA0001140044B80220A41111C1A5C1143195452
:100DB00000BDC04659040010F0B55B18DBB216E068
:100DC0008425CC086C4307270F40802504193D413A
:100DD000EFB2A6189C4605E0064BE5182B780134C7
:100DE0003B432B70B442F7DB01316346C9B29942F1
:100DF000E6D3F0BD59040010F0B589B00591069214
:100E00001C1C5D68DB78834202D22478039444E0A2
:100E1000A378234AC01A0023954209D14300181829
:100E200003234519039309E02A7801330232AD18F0
:100E30008342F9DB69782B7803910235EB180026A1
:100E40000493019625E0082F05D1049A954224D0F9
:100E50002E7800270135F30706D5029A069B0798DE
:100E6000D118C9B2FFF792FF0299761001310291B1
:100E7000013707E0002202920199059A08278B1892
:100E8000DBB20793637802999942DCDB019A013265
:100E90000192019B03998B42ECDB039809B0F0BDF2
:100EA000274E0000F0B585B0061C0C1C029203937F
:100EB00001F052FC00250190832708E0705D211CA1
:100EC000029A039BFFF798FF013024180135A742CF
:100ED00002D3019B9D42F1D305B0F0BD30B50C4C5F
:100EE0000021012204230D5D854203D11801024334
:100EF000D0B20BE0013B002B04D10132092A00DD06
:100F00001A1C042301312829EDD1002030BDC04630
:100F1000D455000000B50F23020918408000031FBC
:100F200000D52833002B0EDB511E03208842804160
:100F30004042002807D1242B06DC04218A1A0349E9
:100F4000CB18985C00E0002000BDC046D4550000DE
:100F500070B5064E051C0024A05D054B291CC01869
:100F6000013400F0CFFC0A2CF6D170BD1056000001
:100F700000400440F8B50E4B1B68002B17D1102021
:100F8000FFF7E6FF0B4C271C143725786678281CE2
:100F9000311C002200F044FC0234281C311C0122C8
:100FA00000F08CFCBC42F0D1014B01221A60F8BD6C
:100FB00034020010FC550000F8B50C4C271C143707
:100FC00025786678281C311C012200F029FC0234A7
:100FD000281C311C002200F071FCBC42F0D1002022
:100FE000FFF7B6FF024B00221A60F8BDFC55000067
:100FF0003402001038B5041CFFF7BCFF002C09D0E8
:1010000007210122022000F00BFC104B80211A68FE
:101010008A431A6000200B2100F026FC01250028DD
:1010200005D000200B2100F01FFC45424541002C5B
:1010300009D007210022022000F0F2FB034B80219F
:101040001A680A431A60281C38BDC046FC3F02508B
:10105000F0B589B000230490012005910693079311
:10106000FFF7C8FF051E02D01823069301250021B3
:101070002A4C019120786178012200F0D1FB207880
:101080006178002200F01AFC0327254E22E0327816
:101090007378101C191C0292039300F0E5FB0028E2
:1010A0000BD03078717800F0DFFB002805D0029873
:1010B000039900F0D9FB002807D10199194AAB0028
:1010C0008A5C183369465A500135019A013F013252
:1010D0000192023EEB0F00210122AA424B41DBB2FA
:1010E0008B4201D08F42D2DA20786178002200F062
:1010F00097FB20786178012200F0E0FB0A4B023474
:101100009C42B7D1281E06D0069B0499059A0B6015
:10111000079B0120136009B0F0BDC046FC550000DC
:10112000D2550000D45500001056000008B501202B
:10113000021C0B2100F074FB01200B21002200F0A7
:10114000BDFB03200221012200F06AFB03200221E3
:10115000002200F0B3FB08BD37B5234B10211A68FD
:10116000051C8A431A60214B8022196892010A43A8
:101170001A6001200B21002200F052FB01200B21FC
:10118000002200F09BFB1A4B9F211A68194C8A43DE
:101190001A601A6818491A60184B186803F018FD8D
:1011A0008023000218432A1C20600221032000F043
:1011B00085FB142000F068FD2368FF229343236021
:1011C00023680F4A134323600E4B1A680192019A59
:1011D000002AFADA22680C4B13402360FFF7A6FFBF
:1011E00001980004800D3EBD388204408080044098
:1011F0009840044000C0014000093D00680500100F
:10120000800000012CC00140FFFFFFF810B50C4C1E
:101210002068002813DA00202060FFF79DFF0A28CD
:101220000ADC0120FFF798FF0138C023FF385B007C
:10123000984201D801232360FFF778FF206810BD92
:101240001C00001008B5FFF7E1FF011E08D00120C7
:10125000FFF782FF011E03D0024803F0B9FC011C16
:10126000081C08BD50BB120008B5FFF7CFFF0028CF
:101270000AD0FFF7E7FFFA22031C0021C00FD200BB
:101280009A424841014B186008BDC0463802001020
:1012900008B5074B02221A60064BA2221960064BC2
:1012A0001A70A32258709A7000F0ECFE08BDC04678
:1012B00094050010700500108405001008B5064B59
:1012C00002311960054B00221A60054BA2221A70E8
:1012D000587000F0D7FE08BD94050010700500108E
:1012E00084050010F8B5074F051C0E1C0324281CAC
:1012F000311CFFF7CDFFB84202D0013C002CF6D1E3
:10130000F8BDC04601010000F8B5074F051C0E1CD2
:101310000324281C311CFFF7D1FFB84202D0013C46
:10132000002CF6D1F8BDC0460101000070B50E4B8F
:101330001B68002B16D00D4BFF24151C25409E78F2
:101340009D70150A2540DE78DD70150C2C40120EBC
:101350001D791C715C795A71FFF7D6FF831EFF3B24
:101360005A425341181C70BD3C0200108405001005
:10137000F8B5164C2468002C25D0154CFF25161CFA
:101380002E40A778A670160A2E40E778E670160C55
:101390002E402779120E2671667962711A1C2A4036
:1013A000A679A2711A0A2A40E679E2711A0C154050
:1013B0001B0E227A2572627A6372FFF7A5FF841EE4
:1013C000FF3C63425C41201CF8BDC0463C0200105B
:1013D0008405001008B5064B1B68002B05D0FFF7ED
:1013E00081FF831EFF3B5A425341181C08BDC04673
:1013F0003C02001008B5064B1868002807D00220F0
:101400000721FFF76FFF0238FF384342584108BDFC
:101410003C02001008B5064B1868002807D00220CF
:101420000721FFF771FF0238FF384342584108BDDA
:101430003C02001010B50120011CFFF753FF0B4BBD
:1014400098420ED10A4B012119600A4B1C782307E0
:1014500009D0094B032222409A70081CFFF754FF61
:1014600001E001246442201C10BDC04601010000BF
:101470003C020010740500108405001008B5FFF749
:10148000D9FF02200121FFF72DFF0A4B98420FD10F
:10149000094B1B787F2B06D9842202200721520496
:1014A000064BFFF765FF09200421054AFFF73EFFC1
:1014B00008BDC046010100007405001003011400BE
:1014C0008080808010B500280DD0264B80211A68BE
:1014D0008A431A60244A012311681942FCD0234B25
:1014E00003221A6001E0214B1860214B01220021E8
:1014F0001A6019601A6019681142FCD01D4B012254
:101500001A601D4A802114684902214311601A1C87
:10151000002804D1134B8024196821431960174B0C
:10152000196888421CD01860002801D0144800E0D7
:101530001448116803F0FEFA134BFA211860890071
:10154000041C03F045FB1E235843104BC8211860B0
:101550004901201C03F03CFB0D4B186001F02CF9F5
:1015600010BDC046388204400C80044070800440A6
:101570007480044078800440808004402000001083
:10158000006CDC02001BB700680500106405001049
:101590006C05001008B500F035F9134B00211A68EE
:1015A000120B12031A60114B1A68120B12031A6005
:1015B0000F4B1A68120B12031A600E4B1A68120BAB
:1015C00012031A600C4B012219600C4B1A6019604F
:1015D0001A6019681142FCD0094B23221A600120BD
:1015E000FFF770FF08BDC04600800050008001502A
:1015F000008002500080035040800440448004403A
:101600000880044070B50F490F4801F04DF80F48AD
:1016100001F04AF80E4E0F4D00242B196159DA687B
:10162000301C0A4B143401F03FF8B42CF5D10A48B1
:1016300001F03AF800F044FB011C084801F034F8CE
:1016400070BDC046044D00001A5600006C560000E4
:101650002C56000024000010375600005956000098
:10166000F0B53C4B8BB01D68002D3AD03A4B029040
:101670001B6801209B685DE001342378202BFBD0A0
:10168000002B3AD0B30008336A469C500136FF2D38
:1016900001D135E001342378202B01D0002BF9D182
:1016A000202B02D1002323700134012E1BD12A4F9D
:1016B0002A4B0A223B6001923D1C09E02B680298EC
:1016C000196801F06BF8002808D02B6814332B60E0
:1016D000019B013B0193002BF0D132E03B681D7967
:1016E00001E0041C2E1C2378002B06D000230722C7
:1016F000B2425B41DBB2002BBFD1002E1CD000E018
:101700000025154C022E05D10398154901F046F825
:10171000002801D0AE420AD823681248D96800F0E8
:10172000C3FF23681048196900F0BEFF04E0236876
:10173000F0B29B6802A99847064B1B68002B07D1A3
:1017400003E00198011CFFF75DFF084800F0ACFFC3
:101750000BB0F0BD4003001048030010240000103F
:101760006656000068560000084E00006F560000E4
:1017700038B5041C154D0A2808D002D808281CD1F9
:1017800010E00D2802D07F2817D10BE02B68002233
:101790001A700F4800F088FF0E4C201CFFF760FF06
:1017A0002C6012E02A680B4B9A420ED90A48211C81
:1017B00000F07AFF2B68013B06E00748211C00F08F
:1017C00073FF2B681C7001332B6038BD440300107D
:1017D0006C560000400200107B56000008B503E084
:1017E00000F000FEFFF7C4FF00F01EFE0028F7D156
:1017F00008BD0000014A024B1A6070474002001009
:1018000044030010044B40211A680A431A60034B3A
:1018100001221A707047C046808004404C030010BB
:1018200070B50E4B061C1B780D1C141C002B01D12F
:10183000FFF7E8FF013E022E03D8094BB600F3582C
:1018400000E0084B1A68012C03D1AC4014431C6023
:1018500003E00124AC40A2431A6070BD4C030010A9
:10186000485700000080005038B50F4B051C1B780E
:101870000C1C002B01D1FFF7C5FF0020032D11D850
:10188000281C012303F042F902040608074A04E079
:10189000074A02E0074A00E0074A1068A3401840E0
:1018A000431E984138BDC0464C030010FC3F005019
:1018B000FC3F0150FC3F0250FC3F035070B50E4B03
:1018C000061C1B780D1C141C002B01D1FFF79AFF7E
:1018D000013E022E03D8094BB600F35800E0084B36
:1018E0001A68012C03D1AC4014431C6003E00124AE
:1018F000AC40A2431A6070BD4C0300105457000066
:10190000FC3F005038B5084B041C1B780D1C002B05
:1019100001D1FFF777FF23681822934323602368E0
:101920001D43256038BDC0464C0300101F234209EB
:10193000184001238340181C014B9200D05070477F
:1019400000E100E01F234209184001238340181CD6
:101950002032024B9200D0507047C04600E100E0B8
:10196000054B3F221A60054B01221A60044B4021AF
:101970001A688A431A60704724800440D880044063
:101980003882044008B5044B40211A688A431A6023
:10199000FFF7E6FF08BDC0463882044008B500F0F6
:1019A00037FBFFF709FB0A480021FFF7ABFF0948A7
:1019B0000021FFF7A7FF08480021FFF7A3FF074812
:1019C0000021FFF79FFF06480021FFF79BFF08BD9E
:1019D0000840044000400440AC400440144004402F
:1019E0001C400440F7B5071C0D1C72B6FFF7D6FF6C
:1019F000504B1A68504B1A60002F01D04F4B00E03B
:101A00004F4B504A042113604F4B504C1A680A4305
:101A10001A6000232360A90720D04D4B4D4A196856
:101A20000A401A60AA0711D52268EC235B01134310
:101A300023600720FFF77AFF0820FFF777FF0A20CF
:101A4000FFF774FF0C20FFF771FF04E0226880238A
:101A50001B01134323600B20FFF768FF002F58D0B2
:101A60003D4B00251D603D4B3D4E1D603D4B301CE8
:101A70001D603D4B291C1D60FFF744FF281C0921F8
:101A80002A1CFFF7CDFE281C09212A1CFFF716FF90
:101A9000364B80211A680A431A6033680722934341
:101AA000336033680222134333607B01DF1BB801CC
:101AB000C71B0A21B80003F03DF82D4B0322186024
:101AC0002C4B09201D602C4B1A602C4B2C4A19689A
:101AD0000A401A601A6880210A431A60FFF726FF3D
:101AE0001B4A802311689B00194311602268022160
:101AF0001343244A236001231360234A1160234ABD
:101B0000154913601560136010681842FCD001235A
:101B10000B601F4B012252421A601E4B1A68019241
:101B200062B630BFC046019A1B689A4200D130BFEE
:101B3000F7BDC0463882044034820440BF1800001C
:101B4000FF1800003082044010ED00E004820440E1
:101B5000008204407FE2FFFF04C000400400014017
:101B600064400440044001400480014080800440FF
:101B700018C0004008C0004014C000403CC00040F5
:101B80000FF0FFFF788004407080044074800440B0
:101B9000088204405003001008B5FFF723FF08BD7A
:101BA00008B5012000F0E4F908BD000008B5164BA7
:101BB0001868FFF787FC0720FFF7C4FE0820FFF72F
:101BC000C1FE0A20FFF7BEFE0C20FFF7BBFE0B2074
:101BD000FFF7B8FE0920FFF7B5FE0C4A002313609B
:101BE00001210B4A494211600A4A13600A4A1360F4
:101BF0000A4B01221A60FFF7D3FF094B1A68013222
:101C00001A60C046C04608BD20000010048204408F
:101C10000882044004C000403CC0004000C00040B6
:101C20005003001000B5084B1A68013203D1074A6F
:101C30001168013111601A6801321A60044B1A6888
:101C400001321A6000BDC046600300105C03001042
:101C50005403001000B5074B98420AD8064A0023E7
:101C60001360064A01381060054A1360054B0722CD
:101C70001A6000BDFFFFFF006003001014E000E0E9
:101C800018E000E010E000E000B50C4A13680028FE
:101C900000D10120C1438B4204D809E01168814280
:101CA000FCD301E0591C081811689942F6D203E0F0
:101CB0001168C91A8142FBD300BDC0466003001001
:101CC00010B5064BFA211868054B89001C6802F014
:101CD00031FF044B5C43201810BDC0466003001068
:101CE0005C03001037894100034B01221A60034B4B
:101CF0001A6801321A60704700C000406403001087
:101D0000034B01221A60034B1A6801321A607047B4
:101D1000000001406803001000B5002803D1044B07
:101D200001221A6003E0012801D1024B186000BDB6
:101D300004C000400400014000B5002802D1044B5B
:101D4000186004E0012802D1024B00221A6000BD95
:101D500004C000400400014000B5002801D1054B3B
:101D600002E0012804D1044B1A6802210A431A60D8
:101D700000BDC04604C000400400014010B5002969
:101D800000D1134900280DD1124B80241A68224338
:101D90001A60114B03221860104B1960104B1A6027
:101DA000620211E0012811D10A4B8022186852000A
:101DB00002431A600B4B00221A600B4B032219607E
:101DC0000A4B1A6080229202094B1A6010BDC0466D
:101DD000FFFF0000808004406403001018C0004032
:101DE00014C00040680300101800014014000140B6
:101DF00000E100E010B5514B1A6801321A60504BF7
:101E00001A68504BD2B2302A53D00ED8182A34D088
:101E100005D8082A16D0102A00D08CE020E0202A0D
:101E20005AD0282A00D086E029E0482A54D004D885
:101E3000382A47D0402A7ED148E0502A55D0582A27
:101E400079D168E0404A0021116011683F48445C44
:101E50003F4801310460116028221A60012242E0EB
:101E60003C4A00211160384A38481168445C3848BF
:101E700001310460116028225EE0334A05E0324AF5
:101E8000354910680968884206D211682F48445CB9
:101E90002F48013104604DE0304A11688022D2059C
:101EA000002901D0202145E02D492E48086010214D
:101EB00040E08022D2051021116008221A608122A0
:101EC000520010E082214900254A33E0234A11687C
:101ED0000422012919D11CE08022D20510211160B1
:101EE00008221A60204A1E4B26E01A4A1848116838
:101EF00004681E48E4B24454013111601068174A66
:101F0000116804220139884203D28021C9050A6080
:101F100011E01A600FE00F4A0D4811680468134879
:101F2000E4B24454013111600E490D4A116080221F
:101F30001021D205116008221A6010BD780300102C
:101F400004000040180000407403001084050010D5
:101F5000080000406C03001094050010700500108C
:101F6000700300100101000003010000740500105F
:101F700010B51B4B02211A68041C0A431A60194B46
:101F800020211A680A431A60174B18491A680A4038
:101F90001A601868012210431860154B1868014038
:101FA000196019680A431A60124B6C221A60124BAE
:101FB0001249186802F00CFE114B1860114B1860A2
:101FC000022C02D1104BA0221A60104B8022120268
:101FD0001A6080234022DB0501201A6010BDC04634
:101FE000048004408080044030400440F8FCFFFF3F
:101FF000344004401800004068050010400D030004
:1020000014000040100000400C00004000E100E01F
:1020100008B5164B80221202DA67154B6C221A6043
:10202000144B154A1968002011401960196819608D
:10203000124B19680A401A601A6804211A600122BA
:10204000FFF7EEFB002004210122FFF737FC002000
:1020500005210122FFF7E4FB012200200521FFF703
:102060002DFC074B00221A6008BDC04604E100E0C9
:102070001800004030400440F8FCFFFF34400440AA
:102080000480044000B51649164A002313600B6013
:10209000154920200B608021C9050860134900E024
:1020A00001331068012802D08B42F9D102E00F49B8
:1020B0008B4210D10E4B8021C905102208200A60E6
:1020C000186080235B010868104008D0013B002B9A
:1020D000F9D1181C03E01368FF2BFCD9106800BD70
:1020E0006C0300107003001074030010FF0F000059
:1020F00018000040034B01221A60034B1A6801329A
:102100001A607047004001407C03001000B50028B1
:1021100003D1044B01221A6003E0012801D1024BD4
:10212000186000BD044001400480014000B5002853
:1021300002D1044B186004E0012802D1024B0022B6
:102140001A6000BD044001400480014038B5184BBE
:1021500001251D60174B1A6852191A60164B1A6830
:10216000002A23D01A68154C013A1A601A68002A0E
:102170000DD02268281C291CFFF7A0FB2368281C0F
:10218000EB1A236022680221FFF798FB0EE01B6820
:10219000281C23602268291CFFF790FB281C22685A
:1021A0000221FFF78BFB281CFFF7C0FF38BDC0469C
:1021B0000080014084030010800300108803001099
:1021C00000B5002801D1054B02E0012804D1044BE1
:1021D0001A6802210A431A6000BDC046044001404B
:1021E0000480014010B500280FD1124B80221C68DA
:1021F000920022431A60104B032218600F4B1960A3
:102200000F4B1A608022D20211E0012811D1094B34
:1022100080221868D20002431A600A4B00221A601A
:10222000094B03221960094B1A6080221203084BE4
:102230001A6010BD808004407C03001018400140EB
:1022400014400140840300101880014014800140B4
:1022500000E100E008B5184B1A680E231340062B66
:102260000DD1164B9E221B68DBB2134204D0144AD8
:102270005360144B1B681EE0D9071CD501E0042BEA
:1022800005D1104B1868C0B200F0BDF813E00C2B5C
:1022900006D10B4B8022596852000A435A600AE06B
:1022A000022B08D1054B1A68054B910601D5002277
:1022B00000E001229A6008BD0880004014800040C0
:1022C0008C03001000800040004870478C03001011
:1022D00073B52E4C2E4B8022002192030191061CD7
:1022E000DA67201C902200F017FA019B0725A360F3
:1022F000284B294C1A68AA431A6019680122114315
:102300001960264B1968A9431960196811431960AF
:10231000234B80211868490101431960214B1A6041
:1023200083222260204A12681968204B18685043A3
:1023300002F000FC311C000902F0FCFB1C4B1022D7
:102340001C491A60030A1C4A0B60C0B203231060C8
:1023500023601A4B1D601A4B1868019060201C689E
:102360000440602CFBD102E01468019400E00120DD
:102370001C680442F8D1054B01221A70114B8022CF
:1023800092031A6005230B6073BDC0468C030010D6
:1023900004E100E0A44004400C800040A840044058
:1023A00080800440988004407880044068050010D4
:1023B00028800040048000400080004008800040E9
:1023C0001480004000E100E000B5044A20231168B9
:1023D0001942FCD0024B186000BDC046148000407A
:1023E0000080004008B5FFF76FFF827B031C821856
:1023F000D07B9A7B0132D2B29A7352B2002A01DAB0
:1024000000229A7308BD10B5041CFFF75DFF437BE3
:10241000C318DC73437B0133DBB243735BB2002B25
:1024200001DA0023437310BD08B5FFF74DFF827B2F
:10243000437BD01A431E984108BD30B5002402E00A
:102440000570013401301D5D002DF9D1121B131CE4
:1024500002E00170013B0130002BFADCD043C017D1
:102460000240A01830BDF8B5051C0F1C1E1C541EE0
:10247000092B01D800240FE0181C0A2102F05AFB96
:10248000221C031C391C281CFFF7EDFF041C2D180F
:1024900005E02F7001340135013A002AF9DC301CC7
:1024A0000A2102F08BFB30312970601CF8BDF8B5B1
:1024B0000C1CD9175F18061C4F40551E092F12D946
:1024C000381C0A21002B03DA02F034FB434202E0FD
:1024D00002F030FB031C211C2A1C301CFFF7E7FF15
:1024E000041C351813E0002B00DA951E002201E0D1
:1024F000B4540132A91A0029FADCEC43E4172C4049
:102500003519002B03DA2D232B7001340135381CCB
:102510000A2102F053FB30312970601CF8BD73B5FD
:10252000069E041C1D1C3009531E00280AD0009072
:102530001A1C201C2B1CFFF7F2FF241805E0217049
:1025400001300134013A002AF9DC0F231E40092E24
:1025500001D8303604E0002D01D0373600E0573680
:102560002670013076BDF0B585B0041C0F1C002824
:1025700001D00021017000256BE0252903D02170D6
:102580000132013405E05178252904D1217002324D
:10259000013401355DE0302903D00132029220215F
:1025A00001E002320292029E9C4632782D3A50425D
:1025B0004241B6180296002205E00A235A438218C7
:1025C000303AD2B201363078031C303B092BF4D9B3
:1025D0000296AE186346BE4201D97A1BD2B2692870
:1025E0000ED006D863282CD0642809D058283ED1B4
:1025F00019E075280AD078280FD0732837D11AE04F
:102600001E1D201C1B68FFF752FF04E01E1D201C2E
:102610001B68FFF728FF331C17E01E1D1B68201CDA
:102620000093002304E01E1D1B68201C009301235F
:10263000FFF775FFEFE71E1D201C1B68FFF7FDFE6F
:10264000E9E71A68012022700433029A2418013243
:102650002D181178BD4201D200298ED10023BD4230
:1026600001D2237005E0013C2370013D01E001250A
:102670006D4205B0281CF0BD10B50C1C131C642164
:10268000221CFFF770FF10BD00B5031C9BB00A1C95
:1026900001A8191CFFF7F0FF632800DDFEE701A881
:1026A00000F0B0F81BB000BD0FB407B504A901C914
:1026B0000191FFF7E9FF03B008BC04B018470EB45E
:1026C00003B503AA02CA0192FFF7D6FF02B008BC05
:1026D00003B0184770B50323041C184205D10D1C24
:1026E000041C194201D1934201D3002311E0131CB1
:1026F00040CD043B40C4032BFAD8141FA408013476
:10270000A400032309191A400419EEE7CD5CE5542F
:1027100001339342FAD170BD30B50B040D061D4351
:102720000D430B021D430323041C93420DD2184298
:102730000BD1131C043B20C4032BFBD8141FA4088B
:102740000134A40003231A400419002301E0E154DA
:1027500001339342FBD130BD00B5002300E00133CB
:10276000C25C002AFBD1181C00BD00B5031C01E0AF
:10277000013101330A781A70002AF9D100BD30B551
:10278000031C002406E01D5D085D281A05D10134F4
:10279000002D02D09442F6D1002030BD00B502E0F9
:1027A0000130002B06D00A78037801319342F7D02C
:1027B000981A00E0181C00BD08B5094BFA211868EA
:1027C000890002F005FAFFF745FA96200002FFF7AC
:1027D0007FFD0120FFF7CCFBFEF750FE08BDC04691
:1027E0006805001008B5FEF7D5FEFFF70BF8FFF7F8
:1027F000C9F8FEF775FAFEF761FAFFF7DDFFFEF79D
:10280000F9FF08BD10B5041C02E00134FFF7DCFD40
:1028100020780028F9D110BD70B5054E051C0E2496
:10282000013C295D301CFFF73FFF002CF8D170BD43
:102830006057000038B51648FFF736FF154C201CCE
:10284000FFF7EAFF144D4221281CFFF72DFF201C43
:102850000E30FFF7E1FF4321281CFFF725FF201C66
:102860001C30FFF7D9FF0D48FFF71EFF201C2A3050
:10287000FFF7D2FF281C4E21FFF716FF201C38302F
:10288000FFF7CAFF616D0648FFF70EFF38BDC0466F
:1028900063570000A405001069570000705700003E
:1028A0007657000003110A2253430F2210401818D4
:1028B000704738B50A21041C02F08AF90A21050183
:1028C000201C02F0DBF9281C084338BD08B5C122E2
:1028D00052000E200221FEF729FD024B01225A71FF
:1028E00008BDC0469805001010B5084C6379002B50
:1028F00001D1FFF7EBFF23790C221A43A3790120C2
:102900005B001A43011CFEF711FD10BD9805001075
:1029100010B5074C2379002B08D16379002B01D126
:10292000FFF7D4FF01232371FFF7DEFF10BDC04680
:102930009805001008B5054B1A79002A05D0002229
:102940001A711A72DA70FFF7CFFF08BD98050010F0
:1029500010B501210220FEF73DFD064B041C18783E
:102960007F231840FFF79EFF034B5870DC71201C3B
:1029700010BDC046740500109805001008B5064B40
:10298000064A1B6864201168584302F021F9632845
:1029900000DD632008BDC04654030010580300103A
:1029A000014B01229A70704798050010024B0022DB
:1029B0009A701A727047C0469805001008B5FFF764
:1029C000C7FF094B094A9978002908D0197A0129CB
:1029D00001D8013103E010680549086000E0197270
:1029E0000021D970116008BD980500105403001033
:1029F0005803001008B5FEF71DFD0C23184003D046
:102A0000024B1A781043187008BDC0469805001094
:102A100010B5FFF7EFFF044C23785A0701D5FFF7F5
:102A2000CDFF0023237010BD9805001008B50020CD
:102A3000FEF7E0FA002801D0FFF7EAFF08BD00002A
:102A400010B5054C0023E371FFF7F0FFE379002B8D
:102A500001D1FFF77DFF10BD9805001008B50948AA
:102A6000092102F017F9084BFA22D2001A80FFF769
:102A7000E7FF064B00221A60FA22054B92001A600B
:102A800008BDC04698050010A205001054030010B0
:102A90005803001008B5FFF7C9FF002008BD08B5AE
:102AA000FFF748FF08BD000070B51D4C1D4B2268A4
:102AB0000E1C1A40111CFF231940051C20782170A0
:102AC000110A194060786170110C1940A078120E3B
:102AD000A170E178A188E270134AA0790A401340FE
:102AE0002179120A237163796271FFF7DBFE0F4BC4
:102AF0001B88C01828806079FFF7D4FEA870E078A2
:102B0000FFF7D0FEE870A078FFF7CCFE3070607859
:102B1000FFF7C8FE70702078FFF7C4FEB07070BD7C
:102B2000740500107F7F3F3F071F0000A2050010C3
:102B3000F0B58DB0061CFEF75DFC002804D1301CFA
:102B40001349FFF7BCFD20E00AAC0BAD201C291C8B
:102B5000FFF7AAFF23880693A37807932B78E778DB
:102B600008936B7809930B4BAC78187900F04EF909
:102B7000089B04900193099B301C02930649069A16
:102B8000079B00970394FFF79AFD0DB0F0BDC04678
:102B9000825700007405001087570000F7B50192B6
:102BA00004880D1C061C6421201C02F007F8114B40
:102BB0008FB2E41B1C80A878FFF77BFE0E4CA07040
:102BC0006878FFF776FEE0702878FFF772FE2071D4
:102BD000F078FFF76EFE6A4612796071A271B078E4
:102BE000FFF767FEE071381CFFF763FE2072FEF707
:102BF00011FCFEBDA20500108405001008B5021EE0
:102C000000D0202200200121FEF790FB08BD38B53E
:102C1000041C01200D1CFFF7F1FF201C00F01EF921
:102C2000072102F02BF8201C0A1C291CFFF7B6FF15
:102C300096204000FFF728F80020FFF7DFFF38BD9F
:102C400073B5061CFFF784FE00283AD01D4D6C7842
:102C500006E00A20FFF718F8FFF77AFE002830D0C8
:102C60006B78A342F5D0FEF7C5FB002829D001A957
:102C70006846FFF719FF684600F0F0F8051C01A848
:102C800000F0CCF8104B84199C420DD9E3170122B7
:102C90001343ED18281C694600F012F9002C01DAE4
:102CA0000A4B00E00A4BE418201C01A900F0BFF811
:102CB000281C072101F0E2FF68460A1C01A9FFF762
:102CC0006DFF76BD980500107F5101008051010015
:102CD00080AEFEFFC300074A1B1A03339B185878C7
:102CE0001A78000210189A78DB78120480181B06F4
:102CF000C018704740060010F0B58FB0FDF75EFABF
:102D0000394E00230CA80DA90C93FDF7D9F90C9BA3
:102D1000102B23D10220FFF7DDFF344C0315237263
:102D20003F25C3030011DB0E2840E37160710320CF
:102D3000FFF7D0FF03011B0F013BA37103141D40DC
:102D400002127F2318401A4025710721E270A070FB
:102D50000220FEF7B3FAFDF731FA01E0002B3ED175
:102D6000FDF7ACFFFEF746FB021E2ED0204B3F22A4
:102D700099785D7811401F4F03917F231D407C7827
:102D8000FFF7FCFD1C490190039A2B1C04A800943A
:102D9000FFF795FC04A814210022184BFEF782F8D7
:102DA0000020FEF727F9002801D0FFF731FE0821A7
:102DB0003A780423019104A811490093FFF77FFC9E
:102DC00004A8012109220F4B02E00F480B4B1E21E2
:102DD000013EFEF767F8FDF77BFF002E91D1FDF76E
:102DE000EDF90FB0F0BDC046F049020084050010B7
:102DF0007405001098050010A65700000000001090
:102E0000BA57000014000010CE57000007231840E6
:102E1000014B8000C0587047D800001002783C2356
:102E20005A4341785218534382789818704738B5FE
:102E30000D1C3C21041C01F021FF201CA9703C2129
:102E400001F0C6FE3C2101F019FF6970E121201C50
:102E5000090101F0BDFE287038BD000070B583780F
:102E60000221002299425241048896214901051C01
:102E700064180C20A41A42439B18033B9920584322
:102E80000521023001F0A4FEE3001B19DB001B1931
:102E90009E009B196421C618A210201C4942B61836
:102EA00001F096FEC82136184900201C01F090FE62
:102EB000024B3018C018EB78C01870BDD382FFFFEA
:102EC00070B51E4B0C1CC5181D4B8000C0181D4949
:102ED00001F07EFE43001818C617B60F3618B6105C
:102EE000AE19B600953E301C174901F0C7FECD174C
:102EF000AD0F6D18AD10AB005D190235281C99217E
:102F000001F0BCFE081C052101F062FE0130E070FA
:102F10009921281C01F05CFEC51CEDB2A570301C87
:102F2000094901F055FE094B0C21C6180E20401B23
:102F300001F04EFE3618268070BDC04679050000AF
:102F4000652F0400B13A0200B505000094EDFFFFC3
:102F500030B5F8238A01DB0013404A05920E134373
:102F6000F8221202114019430A235943CA10831848
:102F70001C1CEB345D782478EA336C401B78240207
:102F80001C43835C201C58400723194008418005DE
:102F9000800D30BD7047000008B5054B011C9842FC
:102FA00001DD044BC1180448EA38FFF7D1FF08BD22
:102FB000FF17000000F8FFFF1358000008B5401885
:102FC000511A013101F066FE08BD08B58018891854
:102FD0009A1A0132FFF77EFB08BD000010B5CB0046
:102FE000591A074B0F22C9180023CC5C14400470F7
:102FF000CC5C0133240944700230072BF5D110BD9D
:103000004006001010B5CB00591A064BC918002312
:103010004278047812012243CA5401330230072B4C
:10302000F6D110BD4006001030B5B14B87B0D96E57
:10303000B04D4A1E91416A46D175A96A1A1CC8064C
:10304000400F0138062807D801F060FD040C1F125C
:1030500017191C00022409E05A6E16329200D35848
:103060001C1C15E05B6E16339B00D45800230FE048
:103070009B6DD46DA3420ADC0AE0022403E00C2419
:10308000032305E00D24231C02E00D24EEE70D24AC
:103090002C6148111F2800D922E16A461732944951
:1030A00001F03EFD2000220028002A002D002F0004
:1030B000380040004400490051005F0067006F0085
:1030C000770085009300A200B400C300D500D300B0
:1030D000E300E600E900F100010105010F01110123
:1030E00013011901081C00E08348191C221CFFF77A
:1030F00065FFF5E08148F8E70A1C0E3203E07E48E0
:1031000009E00A1C1C32081C111C1A1C231C01F0AB
:1031100031F9E5E07948011C0E391A1C231CFFF730
:1031200054FFDDE07448011C0E31EEE70A1C1C322E
:10313000081C111CF1E70A6E1020002A00D00A209A
:103140000A1C0E3206E00A6E1020002A00D00A2067
:103150000A1C1C3200946C46173402900194081C1F
:1031600051E001201070086E1022002844D00A227D
:1031700042E00A6E1020002A00D00A200A1C0E32FB
:103180000EE001201070086E1022002855D00A228F
:1031900053E00A6E1020002A00D00A200A1C1C32BC
:1031A00000946C46173402900194081C78E00A6E73
:1031B0001021002A00D00A21504A68461730019099
:1031C00002910094101C111C1DE00A6E1020002AB0
:1031D00000D00A20494A00946C46111C1734029012
:1031E0001C390194101C0EE0096E01201070102291
:1031F000002900D00A224149684617300190029206
:103200000094081C002201F0BFF869E00A6E10204B
:10321000002A00D00A20394A00946C46111C173449
:1032200002901C390194101C3AE0096E01201070C4
:103230001022002900D00A22304968461730019038
:1032400002920094081C00222AE0012010700A6EED
:103250001021002A00D00A21284A68461730019020
:1032600002910094101C00211AE0009222481CE0F8
:103270000092224819E00A6E1020002A00D00A208D
:103280000A1C1C3206E00A6E1020002A00D00A2018
:103290000A1C0E3200946C461734029001940020F0
:1032A00001F09BF81CE00092081C002104E00D1CBA
:1032B0001C35081C0092291C1A1C231C01F0E8F87C
:1032C0000EE0081C02E00C4800E00C48191C221C0F
:1032D00001F0F7F804E0081C221C191C01F0FCF8AE
:1032E0006B46DA7D024B07B00120DA6630BDC0467E
:1032F000A4050010400D0010B2050010C00500101C
:1033000010B506490B1C88331A68141C1E34A4001F
:103310006050013203210A401A6010BDA40500105C
:10332000054B0320191C88310A68013A02400A60E3
:103330001E329200D0587047A4050010F8B5114D08
:103340002C1C8C3420680130FFF726FE0E4B012226
:10335000D8629F6AAB6E061C02409A4210D1830766
:1033600003D420680230FFF7CBFFFF239B001E40F1
:10337000B601BF10044B8C35374301222F60DA6051
:103380000220F8BDA4050010400D001030B50C4B14
:103390000C489A6A031C8C331C68D3059B0E91055C
:1033A00000D5403B856E921001210A40AA4204D10B
:1033B000E3188C300360024BD960012030BDC04659
:1033C000400D0010A405001008B5084B5A1CD07F12
:1033D0009A1CD27F000112021043DA7F0333DB7F95
:1033E00010431B031843FFF78BFF08BDA405001013
:1033F00038B5FFF795FF064903230F22051C5C181B
:103400001540013325770011072BF7D138BDC04691
:10341000A405001008B5FFF783FF034B01228C338E
:103420001860024BDA6008BDA4050010400D0010C2
:1034300010B5064CA36E002B06D0FFF771FF044BAE
:103440008C3401222060DA6010BDC046A405001053
:10345000400D001010B5064CA36E002B06D1FFF7EF
:103460005FFF044B8C3401222060DA6010BDC0463F
:10347000A4050010400D001008B5104B0022596A39
:103480001A62914214D05969914216DD012906D180
:10349000D969914203D0DA610A2299615A615A6965
:1034A000032A02DD06490120C866013A5A6104E098
:1034B000044B1B68002B00D0984708BD400D00103E
:1034C000A40500101C04001000B5084B5A6A002A1D
:1034D00002D05A69002A07DD9A690F21044B114076
:1034E000D97712110133DA7700BDC046400D0010C4
:1034F000A4050010044B597F9A7F090112020A4368
:10350000197F0A435A677047A405001030B50B1C99
:10351000093B012B0FD8084A00239C18257FC45C67
:10352000A54205D0054B08395A681143596002E09D
:1035300001330E2BF1D130BDA4050010400D001059
:1035400008B508290DD0192913D1427808231A4249
:1035500002D00022027002E00F23037007234370A1
:1035600005E000231A1CC25401330E2BFBD1FFF7D8
:1035700049FD08BD1FB5114B5C6F002802D00F221A
:10358000944304435C67FF2C06DD181C1C300021AB
:103590000D22FFF713FD10E06846211CFFF71EFD0A
:1035A0006846211CFFF7CCFF044A00236C46185DD7
:1035B0009918013308770E2BF8D11FBDA405001010
:1035C00030B5124C0F23656F85B09D430543656789
:1035D000082D19D0FF2D17DC6846291CFFF7FEFCCB
:1035E0006846291CFFF792FF00231A19127F6946CB
:1035F0005A5401330E2BF8D16846291CFFF7A0FF5F
:103600006846291CFFF7FEFC05B030BDA40500107C
:103610001FB50F4C616F082918D0FF2916DC6846CA
:10362000FFF7DCFC616F6846FFF770FF00231A1993
:10363000127F69465A5401330E2BF8D1616F6846E8
:10364000FFF77EFF616F6846FFF7DCFC1FBDC046D9
:10365000A405001010B50D4C631CD87FA31CDB7FA4
:1036600000011B021843E37F1843E31CDB7F1B03AD
:103670001843FFF791FC0F23021C1A402277021116
:10368000134000126377A07710BDC046A405001058
:10369000044B5A6E16329200D258121A51424A41C5
:1036A000DA667047A405001000B5064B5A6E163254
:1036B0009200D1580139D150002901DA0D21D150A1
:1036C00000BDC046A405001000B5064B5A6E163268
:1036D0009200D1580131D1500E2901D10021D15091
:1036E00000BDC046A405001000B5094B5A6E163245
:1036F0009200D2580D2A03D11A1C2932127805E003
:103700009A18507F117F0001021C0A435A6500BDC0
:10371000A405001010B5084B0F245A6E1632920003
:10372000D1585A6D58181440013104770D2902DC24
:103730005B1812111A7710BDA405001030B50F4B9D
:103740005A6E596D16329200D2580D2A07D11C1CA0
:1037500029342478F02008402043586507E0981861
:10376000447F057F24012C435C650B114377034B99
:103770009A180F231940117730BDC046A4050010D8
:1037800008B504480022011C1C390D23FFF71DFC5D
:1037900008BDC046DC05001008B504480022011C25
:1037A0001C310D23FFF711FC08BDC046C0050010F9
:1037B00008B504480022011C1C310D2300F0DAFD7D
:1037C00008BDC046C005001008B504480022011C11
:1037D0000E390D23FFF7F9FB08BDC046CE050010DA
:1037E00008B504480022011C0E310D23FFF7EDFB44
:1037F00008BDC046C005001008B504480022011CE1
:103800000E310D2300F0B6FD08BDC046C005001006
:103810000C4A0023111C46310B70111C47310B70F0
:10382000111C48310B70111C49310B70111C4A31AD
:103830000B70111C4B310B70111C4C314D320B7045
:1038400013707047A405001000B5074A011C04233B
:1038500000208A1804E0D118463109784000084356
:10386000013BF8D200BDC046A405001030B5074AA0
:1038700000238918012206E0CC18051C46341540A7
:10388000257040100133042BF6D130BDA405001083
:1038900038B50020FFF7D8FF084C051C0021207F19
:1038A000FFF7E4FF25770420FFF7CEFF0421051C76
:1038B000607FFFF7DBFF657738BDC046A4050010C9
:1038C00010B50020FFF7C0FF034C20770420FFF75E
:1038D000BBFF607710BDC046A405001010B5054CB5
:1038E0000021207FFFF7C2FF607F0421FFF7BEFFAA
:1038F00010BDC046A405001010B5094C231C8C3324
:1039000018680130FFF748FB064B021CD8620F23F2
:103910001A4022770211134000126377A07710BD7E
:10392000A4050010400D001010B5094C0021201C0A
:103930000D22FFF743FB201C0E3000210D22FFF764
:103940003DFB201C1C3000210D22FFF737FB10BD72
:10395000A405001010B50C4B00211A1C187F1C7810
:1039600001312043187701330E29F7D1936E002BD4
:1039700008D0064B1B690D2B04D1137F111C293174
:103980000B70537310BDC046A4050010400D00100D
:1039900010B50C4B00211A1C1C7F187801312040F7
:1039A000187701330E29F7D1936E002B08D0064B00
:1039B0001B690D2B04D1137F111C29310B7053731C
:1039C00010BDC046A4050010400D00107FB50023B7
:1039D0000C4A0D251C1C1118097F01306E469955A3
:1039E000C60F8542664176420133111C30400E2BD2
:1039F000F1D100236C46185DCA18013310770E2BE5
:103A0000F8D17FBDA405001010B5074B5A6E1632D1
:103A10009200D1585C1801392077D150002901DA81
:103A20000D21D15010BDC046A4050010034A00234B
:103A3000111C943198320B6013607047A40500107C
:103A4000034B012194331A684A401A607047C046FC
:103A5000A4050010044A002313678C321360034B43
:103A60000122DA607047C046A4050010400D001026
:103A700008B59C4B0F20996A9B4A8B1018408911FE
:103A8000013852560E2800D9C5E001F03FF8081160
:103A90001A2327C42EC4C437C4C4C43B3F00002A21
:103AA00000DAB8E0914B9A1840320023937133E06A
:103AB000002A00DAAFE08D4B01209A184032907155
:103AC000A8E0002A00DAA6E0884B9A1840329279E2
:103AD000DA6621E0081CFFF797FF1DE0002A00DAF4
:103AE00099E0101CFFF7D4FD16E0002A00DA92E0FE
:103AF0007E4B596E16318900CA500DE0081CFFF745
:103B00005FFD09E0081CFFF735FD05E0002A00DA3B
:103B100081E0101CFFF75AFF01207BE0734B01206E
:103B20009833186076E0FFF7DFFDF5E7FFF792FFC7
:103B3000F2E7FFF725FEEFE7FFF7ECFDECE76B4B55
:103B400000225A66E8E7FFF727FEE5E7FFF7F6FDF4
:103B5000E2E7664B012058665CE0FFF729FEDBE7F1
:103B6000FFF7CAFE022055E0FFF72EFED4E7FFF76D
:103B70002BFCD1E7FFF734FECEE7FFF7D5FECBE70E
:103B8000FFF736FCC8E7FFF737FEC5E7FFF79CFCF9
:103B9000C2E7564B00221A66BEE7FFF7ABFCBBE755
:103BA000524B0120186635E0FFF740FFB4E7FFF7FE
:103BB0002FFDB1E7FFF744FFAEE7FFF74BFDABE7A3
:103BC000FFF78CFEA8E7FFF733FCA5E7FFF7C2FE7F
:103BD000A2E7FFF775FE9FE7FFF73CFC9CE7FFF7C6
:103BE000D7FE99E7FFF714FE96E73E4B01201862D7
:103BF00010E0FFF741FC8FE7FFF756FD8CE7FFF77A
:103C000047FE89E7FFF760FD86E7FFF703FC83E7E0
:103C10000120404208BD982BBBD03FDC382B98D008
:103C20001EDC1C2B00D184E70DDC0C2B00D175E7CA
:103C300003DC0120002BEDD0EAE7162B00D172E760
:103C4000182BE5D172E7282B00D178E702DC262B70
:103C5000DED171E72C2B00D175E7362BD8D175E773
:103C6000662B00D186E70CDC4C2B00D178E702DC18
:103C70003C2BCDD171E7562B00D175E75C2BC7D11A
:103C800075E76C2B00D17BE702DC682BC0D174E7B1
:103C9000762B00D177E7882BBAD177E7E62B00D1D6
:103CA00097E725DCC82B00D184E70CDCA82B00D1DA
:103CB00076E702DC9C2BABD16FE7B82B00D173E722
:103CC000BC2BA5D173E7D62B00D179E703DCCC2B35
:103CD00000D09DE771E7D82B00D174E7DC2B00D032
:103CE00096E773E7400D001013940000A405001040
:103CF000F32B00D17DE70EDCEC2B00D16FE703DC6A
:103D0000E82B00D084E767E7F12B00D16AE7F22BBC
:103D100000D07DE769E7F62B00D170E703DCF52BD7
:103D200000D075E768E7F72B00D16BE7F82B00D0E0
:103D30006EE76AE738B5184C231C8C331868FFF718
:103D40002BF9E26E154BA2660022E266DA600322CE
:103D50009862251C10401C1C022809D090420AD0F1
:103D6000012802D0FFF784FE07E0FFF7E7FA04E03E
:103D7000FFF75AF901E0FFF709FB00280BDDE368C4
:103D8000002B04D12B1C8C331A6812181A60903542
:103D90002B681B182B6038BDA4050010400D0010C7
:103DA000034B0122DA660F229A775A771A77704707
:103DB000A405001010B5054C0549201C00F06AFF51
:103DC000FFF7EEFF0123636610BDC046A405001097
:103DD0009C0700007047000030B50C4D049C286023
:103DE0000B4801600B490A600B4A13600B4B039AA6
:103DF0001A600B4B0B4A1C600B4B1C600B4B1A6080
:103E00000B4B0C4A13600C4A136030BD4004001089
:103E10004C0400105404001028040010200400106A
:103E2000FC0000107D3E0000400D00101C0400103E
:103E3000D53D00005004001038040010014B1860FC
:103E40007047C0462404001010B5094B1A68191CAD
:103E5000084B002A03D1084C2468226003E01A684A
:103E6000824200DD101C186001230B6010BDC046AB
:103E70002C040010480400102404001013B5002383
:103E800000930193114B124C1A68124B1068196879
:103E9000884202D12368009308E012681A600E4B32
:103EA0001B68002B02D0684601A99847009B23603D
:103EB000002B04D0094A64209361FFF7C5FF009AE4
:103EC000531E9A41064BDA6613BDC0462804001003
:103ED0003C040010F80000104C040010400D0010CD
:103EE000A405001000B5034B1B68002B01D1024A4A
:103EF000136000BD340400102C040010014B4A3341
:103F000018787047A405001038B5164B1A1C983263
:103F10001268002A04D0144B1D6801231D4001E0E3
:103F200094331D68114CA3689D4202D16268002A37
:103F300016D0002D02D1002B0AD111E00C4B1B68CA
:103F4000002B02D06168281C98470023636006E0BC
:103F5000074B1B68002B02D0281C291C9847A56022
:103F600038BDC046A405001030040010400D0010FC
:103F70004004001008B5084B084A196812688A1AEC
:103F80001A6006D5FA2252001A60054B1A680132EF
:103F90001A60FFF7B9FF08BD0001001020040010EF
:103FA00030040010F7B50E1C0E21051C019200F024
:103FB00071FE1A4B03240C279E420FDD09236B73FD
:103FC00001232B7328E0301C0A2100F057FE301C1F
:103FD00029550A2100F0FCFD0134061C002E06D0F4
:103FE000E30F0022A7425341DBB29342EBD1019A87
:103FF000A31A033B2B70621B2B1C01E0195D597344
:10400000013BD1180229F9D10F231C1B002301E029
:10401000013C2B55032CFBDCF7BDC046FFC99A3B86
:10402000F7B50024144F051C261C3B68009601962A
:10403000002B02D0684601A99847009B0134002B51
:1040400000D000240220FCF75AF80C4B1A680C4BE5
:1040500010681968884208D012681A60FFF78AFF52
:10406000002D02D0013D002D03D0032CDDDD012009
:1040700000E0281CFEBDC0464C04001028040010BF
:1040800044040010F7B51C4D9B235B000E1C1B4A1B
:10409000E95C1B4BAC5CEB5C002902D00F221440A6
:1040A00002E08021072449009A225200AF5C154AA1
:1040B000CB1AAA5C3435BA1A80277F00791A00918E
:1040C00007210C1B013210490194FEF7F8FA002376
:1040D0000E4F33704124FF35301CFEF73DFB2A782C
:1040E0006B783018D31A391C221C0134FEF7E7FA1A
:1040F000013D462CF0D1F7BDA405001037010000AA
:104100002F010000350100002394000030940000CE
:10411000F0B5504C051CA0614F4893B0031C94337C
:104120001B68E161002B16D1182D0AD1C32908D1D3
:104130004A4B1B680F2B04D138300E21162200F099
:1041400005F9A369182B04D1E369332B01D100F0E1
:10415000A3F8FFF725FE002D00D00A253D4B9A69F4
:104160005D613F4B1A603F4B1B681A683E4B1A60FB
:10417000FFF7B8FE384D012300222B6701928C35E2
:104180003A4A1368002B1BD0394C2368271C002B9C
:1041900016D01B68374E03E0336898473B681B68AE
:1041A000002BF9D023681A68013A1A60324A136862
:1041B000002B05DD013B1360002B01D1FFF792FEC0
:1041C000FFF7B8FD002801DAFCF742F82B4B019A03
:1041D000204C9A4206D1A26A294B9A4202D10A2067
:1041E000FFF732FEA46A2B68264A0194934203D05B
:1041F000254A934214D104E0FFF786FEFBF7AEFF99
:104200000EE0224C2368002B0AD002A80AA9FFF76F
:1042100039FF236802A80AA998472B6827332B6027
:104220001B4B1B6898470F4B1A681A4B106819688C
:10423000884206D012681A60FFF79CFE0D4B1B687F
:104240009847054B1B6F002B9AD1FFF75DFE13B00B
:10425000F0BDC046400D0010A4050010FC00001089
:104260003C04001028040010F80000102C0400107A
:1042700024040010500400104804001066020000DE
:10428000FB030000790D00003E27000054040010DD
:104290003804001044040010F8B5274C00202368AF
:1042A0001D68FFF7BDFE23681A689542FCD01E68A2
:1042B000FFF776FD214B0A22214C5A6118229A61A0
:1042C00001251522DA615D62231C903300222D3610
:1042D0001A60FFF765FDFF362567174C194D0AE098
:1042E000FFF728FD23682A681968914203D01B68EC
:1042F0002B60FFF73FFE23681B689E42F0D1104DF4
:104300000E4C01262B1C90336662182000211F687A
:10431000FFF7FEFE0C4B381C196800F059FC3835CD
:10432000011C0422281CFFF73DFE1823A361002373
:10433000381C6662E361F8BD28040010400D0010CF
:10434000A40500104404001020040010F0B501245E
:104350000DE005780B1C254006E0C65CED007708F3
:104360003D43C554351C2540013BF6D5013A002A92
:10437000EFDCF0BD30B504E0845C8D5C85548C547A
:1043800001329A42F8DD30BDF7B5099D0AAC2678B6
:10439000089F2C7894461D1C002A0DD118E0634616
:1043A0005B5D4A5DD218131901920024B34201DB10
:1043B0009B1B012443550135BD42F0DD0AE0CA5C78
:1043C00012190024B24201DB921B0124C2540133B2
:1043D000BB42F4DD099B1C70F7BDF7B5099E0AAC22
:1043E0002778089D347800282FD000292AD01E1C59
:1043F0009446002A0ED1013F18E063469B5D8A5D1A
:10440000D21A131B00240192A34201DADB19012402
:1044100083550136AE42F0DD37E0CA5C121B002442
:10442000561C01D13A1C0124C2540133AB42F4DDC5
:104430002BE0D15C49420C1B211E01D0E119012463
:10444000C1540133AB42F4DD1FE000291BD0181C1E
:10445000002A06D10EE00E5C135C0130F31A1C1B1F
:10446000E40FA842F7DD10E0CA5C0133141B0134ED
:1044700062425441AB42F7DD07E0D15C013349426F
:104480000C1B611E8C41AB42F7DD099A1470F7BD1D
:1044900070B5049D01242C70141C002905D10BE07B
:1044A000065D0A5D96420BD101349C42F8DD05E0C1
:1044B000815C002904D101329A42F9DD00232B707E
:1044C00070BD00B503E043185B784354013191425D
:1044D000F9DB0023435400BD00B504E08318013B21
:1044E0001B788354013A8A42F8DC0023835400BDD0
:1044F000F0B5114B1A785B78825C1A4000D04022EC
:104500000E4C0F49231C261C04C32C3600221A60B3
:1045100001240A1C123117785578C75D3D4202D03C
:104520001F6827431F60023264008A42F3D10433BC
:10453000B342EBD10020F0BDF9010010000F0010D4
:104540004501001030B512234B43334A0131D318D3
:104550008A0051181A785C78825C144204D02F4A81
:104560005F245218947054709A78DC78825C1442FC
:1045700004D02A4A7C245218533214701A795C7978
:10458000825C144204D0254A7C245218A332147051
:104590009A79DC79825C144207D0204C5F2264183F
:1045A000251CA235A1342A7022701A7A5C7A825CAA
:1045B000144204D0194A7C245218A03214709A7AFA
:1045C000DC7A825C144204D0144A7C2452185032A3
:1045D00014701A7B5C7B825C144207D00F4C5F2204
:1045E0006418251C523551342A7022709A7BDC7B6A
:1045F000825C144204D0094A2E245218A43214704A
:104600001A7C5B7C825C134204D0044B5918F43151
:1046100027230B70002030BD45010010700D0010E5
:10462000F8B52D4C071C0025201C20214F22FEF739
:1046300073F8002D04D0221C7C23393223701370B0
:10464000231C4F330021013519705034052DEBD157
:10465000214B2D22181C38300270181C3730027084
:10466000A1209A705A7040005F221A541B481A54B5
:10467000A320400019541A4908784978385C01424F
:1046800004D0191C533152330A701A700024211CB3
:10469000381C0134FFF756FF0A2CF8D1114D124E89
:1046A00000242B786A78FB5C1A4201D0315905E06E
:1046B0003059FEF751F80D49091A0A310C480434F3
:1046C00000F0F2FA0235242CEBD10A49084800F038
:1046D000EBFA0520F8BDC046700D00104101000046
:1046E000F90100100401001018010010FB01001076
:1046F000B00E001038940000F0B585B00190FCF7C2
:10470000DDFA00226B4C6C4F0092161C754275410D
:104710006A4A009B5D191368012B02D0022B02D15B
:104720005EE1654F02E0002B00D1CDE0002303AA3B
:10473000537023687F210B405C2B00D198E02ADC6A
:10474000382B00D18EE013DC072B6AD006DC022B5D
:1047500000D193E0062B00D0B6E041E0212B00D140
:1047600084E0232B00D187E01C2B00D0ACE081E05B
:104770004F2B4ED007DC3F2B62D0402B62D0392B21
:1047800000D0A1E064E0542B76D05B2B3FD0502BBF
:1047900000D099E06AE0732B66D010DC662B3AD02B
:1047A00005DC5E2B56D0622B00D08DE062E06F2BD3
:1047B0003BD0712B52D06D2B00D085E02DE0792BB2
:1047C0004AD006DC762B4BD0772B3DD0742B7BD197
:1047D00046E07D2B23D07F2B25D07C2B74D135E078
:1047E00031231370022E4BDD231C083B1B6819403C
:1047F000542908D0032E43D0231C0C3B1A687F2376
:104800001340542B3CD14C2203AB1A7038E03223B6
:1048100035E0332333E0342331E035232FE03623F2
:104820002DE037232BE0382329E039231370062E9F
:1048300026DD231F1B6819404723232920D11EE0B2
:1048400030231CE02D231AE0412318E0422316E018
:10485000432314E0442312E0452310E046230EE0F6
:1048600048230CE04C230AE0502308E0522306E0E2
:104870004F2304E0552302E04E2300E04923137048
:104880003B1C03A8291C0022FCF70CFB23681A061A
:1048900005D5E91D0A4800223B1CFCF703FB2368F1
:1048A000DA0572D5E91D074800223B1CFCF7FAFA2D
:1048B0006BE0C046000F0010080000100802001056
:1048C000A75600004094000023680122134206D03E
:1048D000A818C0B2002107220223FCF76DFA236852
:1048E0000222134205D0A81DC0B200210623FCF706
:1048F00063FA236804210B4205D0A81DC0B202222E
:104900000623FCF759FA236808210B4205D0681CDE
:10491000C0B207220223FCF74FFA2368DA0606D555
:10492000681CC0B2042102220623FCF745FA236862
:104930009A0606D5681CC0B2002102220623FCF7A5
:104940003BFA23685A0606D5681CC0B20421072228
:104950000223FCF731FA23681A0607D5281C093010
:104960000222C0B20821131CFCF726FA2368DA05DC
:104970000BD5EDB2281C0930C0B20B210A35FCF76B
:1049800005FAE8B20A21FCF701FA009B01360C3364
:10499000043400930B2E00D0B8E6124B1B68002B9A
:1049A00005D0114800210922104BFCF77BFA104D6D
:1049B000104E114F0024019A2B78D35C6A781A426A
:1049C00006D0A3009859E15D0922084BFCF76AFA6A
:1049D00001340235092CEED1FCF77AF905B0F0BDAF
:1049E000064FA3E6380200104294000014000010A5
:1049F000040100100C0200103C0100100000001027
:104A000038B5FFF77BFA002814D006240321201CB8
:104A100000F0DEF80321C5B2201C00F02FF9281C9D
:104A2000C9B2FCF7B3F9092C01D10B24EEE701342C
:104A30000E2CEBDDFCF74CF938BD000070B5041C02
:104A4000FFF756FD201CFFF757FE0A4B1B78002B83
:104A50000ED0201CFFF7E4FD074CC8235B00074E77
:104A6000E518211C301C5034FDF71EFEAC42F8D175
:104A700070BDC04658040010700D0010084E0000B4
:104A800000B589B000280ED0FCF7E3F801A8092191
:104A9000FEF7A4FA684612300A21FEF79FFA01A831
:104AA000FFF7CCFF08E0FCF7DCF8044B1B78002B89
:104AB00002D00348FDF7F8FD09B000BD580400100E
:104AC0004494000000B5FEE700B5FEE708B50A4BC8
:104AD0000A4A0B4903E010780132187001338B4207
:104AE000F9D3084B0849002201E01A7001338B42C8
:104AF000FBD3FBF7B7FDFEE7000000109B9400001E
:104B000030020010300200102C0F001002B4714669
:104B100049084900095C49008E4402BC7047C04600
:104B200003B47146490840004900095A49008E44BF
:104B300003BC7047002934D00123002210B48842FE
:104B40002CD301242407A14204D2814202D20901BC
:104B50001B01F8E7E400A14204D2814202D24900DD
:104B60005B00F8E7884201D3401A1A434C08A04280
:104B700002D3001B5C0822438C08A04202D3001B16
:104B80009C082243CC08A04202D3001BDC0822432D
:104B9000002803D01B0901D00909E3E7101C10BC51
:104BA0007047002801D00020C04307B4024802A18A
:104BB0004018029003BDC046D90000000029F0D083
:104BC00003B5FFF7B9FF0EBC4243891A1847C04628
:104BD000002941D010B4041C4C40A44601230022FB
:104BE000002900D54942002800D5404288422CD3F4
:104BF00001242407A14204D2814202D209011B01EF
:104C0000F8E7E400A14204D2814202D249005B00ED
:104C1000F8E7884201D3401A1A434C08A04202D355
:104C2000001B5C0822438C08A04202D3001B9C0896
:104C30002243CC08A04202D3001BDC0822430028F8
:104C400003D01B0901D00909E3E7101C6446002CBE
:104C500000D5404210BC7047002806D003DB00207E
:104C6000C043400801E08020000607B4024802A1CA
:104C70004018029003BDC046190000000029EBD087
:104C800003B5FFF7A7FF0EBC4243891A1847C04679
:104C90007047C04600B5002905D0002301390370D4
:104CA00001300029FAD100BDF8B5041CA30719D1C1
:104CB000231C04CB0F4D104E50199043021C201C96
:104CC00032420FD1181C0B4F04CBD51995433542F6
:104CD00008D1181C074F04CBD51995433542F1D0A4
:104CE00000E001300378002BFBD1FDF73EFD201CD6
:104CF000F8BDC046FFFEFEFE808080802573202523
:104D0000730D0A00444D31355F4D38300053455224
:104D100049414C20434F4E534F4C450072656164EE
:104D200079000D0A4279652E2E2E0D0A004E4F0095
:104D30002573202573202025694D485A00563139A6
:104D400000202025692E2530336956002025735216
:104D50005443004C43443A25303269202D202569C4
:104D600000505245535320454E54455220544F2035
:104D70005341564500444D3431204F4B004241448D
:104D8000204B4559202530327800202D2025303207
:104D90007800444D34310020204552523A20256994
:104DA0000025633120484F5552007475726E65645A
:104DB000206F6E003C52455345543E0D0A0042613F
:104DC00064206E756D6265722E0D0A004241543A80
:104DD0002025696D560D0A000D0A253032782020F5
:104DE0000057616974696E6720666F722064617430
:104DF000612E2E2E0D0A00426164206D6F64656C79
:104E00000D0A00526561642025730D0A0046414970
:104E10004C4544006F6666004C43442064656275EF
:104E2000672025730D0A00000000005C000C000CD8
:104E30007C287C7C447C241048285408000C0038D2
:104E40004400443800201008103810804000101032
:104E500010004000201008384438007C006454489A
:104E60004454281C107C4C542438542004740C28BE
:104E70005428085438005000805000102844282836
:104E800028442810045408384C5C7814787C542842
:104E90003844447C44387C54447C14043844347C86
:104EA000107C007C0020403C7C106C7C40407C08E6
:104EB0007C7C047C7C447C7C14083844787C1468BA
:104EC000485424047C047C407C3C403C7C207C6C2A
:104ED000106C1C601C64544C7C4400081020447C02
:104EE00000080408808080040800784478000708DF
:104EF0000400000000BF01BF010905000007000712
:104F000000070007130A00002000E400FC003F0037
:104F1000E700FC003F002700040F0800000C011E02
:104F200001FF03FF032201E201C2190D00000E0080
:104F30001F0011019101FF007E00FC00FE01130122
:104F40001101F001E0140A0000EE00FF011101114F
:104F500001BF01EE00E00130011001050300000F68
:104F6000000F0A050000F800FE03070701040B0606
:104F70000000000001040707FE03F80F080000000E
:104F8000000A000E001F001F000E000A1109000099
:104F9000100010001000FE00FE00100010001008AD
:104FA0000400000004800780030D070000100010BB
:104FB0000010001000100010080400000000800124
:104FC00080010D07000C000FC003F0003C000F0033
:104FD000030F080000FE00FF01010101010101FFB4
:104FE00001FE10080000000002010201FF01FF01A4
:104FF00000010001100800008601C70161012101C4
:1050000031011F010E010F08000082008301110110
:1050100011011101FF01EE11090000300038002CD0
:10502000002600FF01FF012000200F080000800083
:105030009F011F0111011101F101E10F080000FCA6
:1050400000FE010B0109010901F901F00F08000040
:1050500001000100C101F1013D000F00030F080034
:1050600000EE00FF01110111011101FF01EE0F0817
:1050700000001E003F0121012101A101FF007E0867
:1050800004000000008C018C010804000000048C66
:10509000078C0312090000200070005000D800881F
:1050A000008C010401040111090000480048004877
:1050B0000048004800480048004811090000040169
:1050C00004018C018800D80050007000200D0700FA
:1050D0000002000300B101B9010F0006190D000024
:1050E000F800FC010603FB06FD0505050505FD05A9
:1050F000FF050601FC01F8120900008001F0017CA7
:10510000004F004F007C00F00180010F080000FFFD
:1051100001FF01110111011F01FE01E01109000051
:105120007C00FE0083010101010101018301821164
:10513000090000FF01FF010101010101018301FEDE
:10514000007C10080000FF01FF0111011101110195
:10515000110111010F080000FF01FF0111001100F2
:105160001100110001120900007C00FE0083010102
:105170000121012101E301E20112090000FF01FF09
:10518000011000100010001000FF01FF010A0500CF
:10519000000101FF01FF0101010B060001000101F7
:1051A000010101FF01FF10080000FF01FF013800AD
:1051B0006C00C6008301010110080000FF01FF011F
:1051C00000010001000100010001160B0000FF01B9
:1051D000FF010F003C00F000F0003C000F00FF0159
:1051E000FF0112090000FF01FF010F001C00700009
:1051F000E001FF01FF01130A00007C00FE008301B3
:105200000101010101018301FE007C0F080000FF84
:1052100001FF012100210021003F001E140A0000AF
:105220007C00FE0083010101010101038307FE04EC
:105230007C0412090000FF01FF0121002100710020
:10524000DF008E010001110900008E009F01110195
:10525000110111011101F301E21109000001000126
:10526000000100FF01FF0101000100011109000020
:105270007F00FF008001000100018001FF007F111D
:1052800009000007001F007800E001E00178001F1E
:105290000007190D00000F007F00F001E0017C0005
:1052A0001F001F007C00E001F0017F000F120900C9
:1052B000008301C7016C00380038006C00C701830F
:1052C0000111090000010007001E00F801F8011E8D
:1052D00000070001120900008101C10161013101D3
:1052E00019010D01070103010004040200007F0100
:1052F00009050000070000000000070B064400FF3E
:105300000144004400FF01440B0600008C00120120
:10531000FF032201C40D07820045002500920048CA
:10532000014401820C060000E60019012601C000BC
:105330002001070400000000010002080400000032
:1053400000FE0101020804000000000102FE010B42
:105350000600008800500020005000880B06000066
:1053600020002000F80020002006030000000400B8
:10537000020B060000200020002000200020060371
:105380000000000000010905000080016000180015
:10539000060B060000FE00010101010101FE0804E8
:1053A000000002000200FF010C0600008201410122
:1053B000210111010E010B06000082000101110103
:1053C0001101EE0B060000600058004600FF01408E
:1053D0000B0600009F00090109010901F10B0600FD
:1053E00000FE00110111011101E20B060000010095
:1053F000C10131000D00030B060000EE0011011188
:10540000011101EE0B0600008E00110111011101C6
:10541000FE0804000000008C018C0108040000005C
:1054200000000208010A0500002000500088000466
:10543000010B0600005000500050005000500905BC
:105440000000040188005000200B0600000200014B
:1054500000610111000E0D0778008601320149023A
:10546000390242027C0E07800170004C0043004C60
:1054700000700080010B060000FF011101110111F5
:1054800001EE0B06FE000101010101010101820B89
:1054900006FF0101010101010182007C0C060000F0
:1054A000FF0111011101110101010B060000FF01B3
:1054B000110011001100010C06FE00010101011193
:1054C000019100F2010C06FF011000100010001005
:1054D00000FF010804000000000000FF010704C0F5
:1054E0000000010001FF0E070000FF01180024006A
:1054F0004200810000010C060000FF0100010001D4
:10550000000100010E07FF010C003000C000300058
:105510000C00FF010C06FF01060018002000C0006F
:10552000FF010B06FE000101010101010101FE0B5B
:1055300006FF0111001100110011000E0C06FE0003
:105540000101010141018101FE020C06FF01110070
:10555000110011002900C6010B0600008E00110188
:1055600011011101E20B06000001000100FF010121
:1055700000010B06FF000001000100010001FF0D0A
:105580000703001C006000800160001C00030D0781
:105590001F00600080017C00800160001F0E0783F7
:1055A000014400280010002800440083010D070377
:1055B0000004000800F00108000400030E07810148
:1055C0004101210111010901050103010007000842
:1055D000000A0100181110133831303378717073DC
:1055E000C8C1C0C38881808384848782C5C4C7C280
:1055F00075747772353437321514171202070208A2
:105600000201000301090304020402050305000668
:105610002024282C383C4044484C4669726D776100
:1056200072652025735F5631390D0A00252D313002
:10563000732025732573000D0A5479706520273C6B
:10564000636F6D6D616E643E203F2720666F722030
:10565000706172616D730D0A00557074696D65201B
:105660002575730D0A003F0025730D0A0D0A0056BB
:105670004F5941474552203E3E2000256300486572
:105680006C70004E6F20706172616D73004B6579B4
:10569000207072657373003C6B6579313E203C6B02
:1056A0006579323E202E2E2E0044756D70206D657A
:1056B0006D6F7279004C6F6164206D656D6F7279EA
:1056C0000074004765742074696D6500747300533D
:1056D00065742074696D65003C595959594D4D44A4
:1056E000443E203C48484D4D53533E0074640055A1
:1056F00070646174652074696D65003C6F666673E3
:1057000065745F696E5F6D696E757465733E005494
:105710006F67676C6520646973706C6179206F7561
:105720007470757420746F20636F6E736F6C650096
:1057300062005265616420626174746572792076DA
:105740006F6C74616765000000800150008002503A
:1057500000800350FC3F0150FC3F0250FC3F0350CF
:105760002578000D0A413A2000202025633A2000C8
:105770000D0A4D3A20002020473A20253032780D7E
:105780000A006661696C0025692D253032692D2576
:1057900030326920253032693A253032693A253075
:1057A000326920257300253032783A253032783A34
:1057B000253032692E253032690025303278203A82
:1057C000202569202569203A2025303278004E4F67
:1057D0002052544300253032783A253032783A2529
:1057E00030327800253034782D253032782D253030
:1057F000327820202573004D4F4E005455450057F8
:105800004544005448550046524900534154005302
:10581000554E00A0FB627D7F32122BA40B56F8A1DF
:105820008C674689F47B25E6B8033572687BE7E927
:10583000303584961D543CFCE250275C6A68244F46
:105840007650F45B0109FD4E82D9FD9D098719B29E
:10585000D1D2821B209DDCFF025834688D2A78B992
:1058600011A1547420E5701CB2689E22D5ADF19947
:10587000A848FD5F61E9BA322867B933A8521D8A8A
:105880002E7C1AE734A68F021473922102246380BF
:105890003C1057C93B81A453CC834B30E3D9B54E60
:1058A000CB994F66A4DF92C0377C10787D02D05030
:1058B000E88DAD55AAEF4B1748DD329C2E609960FC
:1058C00029C56F2FF7A16BB4985727777E40E99CC5
:1058D0003809297E26E6C4A4CDB032DDEC049B8ACB
:1058E000AC69CE6D5B587537C847ABC306D05F490E
:1058F0000DF7D3728C03EE6C76DFD40085E167DAA6
:10590000DEB1362AA9690F758DE0ECF01F956ECED9
:105910000253ECA2C7334E1297DAC2337CD765D656
:1059200038BC521223E98259C5C5E5662E4B518910
:10593000A597E6DB6DBCCA66953D05F14033F5647D
:10594000FF55204B0F3868B15398DC78E76126DCAF
:1059500074B3C98658632556EA3B62C7A48FFB7CA3
:1059600073C83776A23A827151C2274FE67FBB8A4D
:105970008BD720AD5ADBE778D301872DDA6CC57B56
:10598000A8873C5B168DD73C99BB9F8CF5A4BFCBF9
:10599000A22DCF3E36C6CB3CB66CC841A93AFC1FFF
:1059A000C68E20D283DE0E67DC71F34A36A26D24E8
:1059B000E1558C90C676296B70E9ED21DF6463FFB9
:1059C000C8E42D7038876CFC4159595B084DCBD821
:1059D0005EE3F04527E204E16D1CBEF4C273E99F6B
:1059E000818CF866229A6D600C56DB65BBB3D91BBF
:1059F000638371A16CBB3B2D60DE0613CAA8F7F868
:105A0000DF3B98C3527A63C3FF931929310A12E02E
:105A10009E98404CF69797F29383A62FCED2DF76CE
:105A2000EBA9F9E65B7DD4F2009011712D81366807
:105A3000593286A5FBF4687C95D1E5D14AAB605319
:105A4000D72FB09BC68DAC47E96EA6C61DBAFCBC6D
:105A50008E6045B0AFC5E7D821FF5590F07798D656
:105A6000D734D300B99C7A8C51905C11666BC60D0B
:105A70006B2CAC8917F1058419F07BCC1F0E039AAF
:105A800087DC289746F848F0FB22F690AB219DB3BF
:105A90001E7EF550CA1BF03ED59E30FFE1AF96CB7F
:105AA000027E43652248F9A8F9BAF9513B8100808A
:105AB0004C09365ACA4820B8C0DC4D72A4F7ACA5D0
:105AC0004A4DED02DE7E4E9E8727BDC8F7A2658A4D
:105AD0004F85D26C685E5A97EABAAE03FB9A76CAD3
:105AE000FB21CED23E12CAADB96C180ADFD78C1C8E
:105AF000359509F52B311BF5881554BD0B44327BC8
:105B0000B65A9392B30828D23E9D1A9A37D6960970
:105B10002464448095841671B26D370247A16E6883
:105B2000119D8BE2CB24A77967DB0338E0D8287D71
:105B3000E1CFC200D6CBCE84DCCEACB6379BFFA47F
:105B400059D0F25F973C9D230293FA87E311C25923
:105B50004BFD55F776B590C9B2C7BBAB784B9CCA25
:105B60004BE8592F21DCD3C937EC5F595C5F17181C
:105B7000F313073590C22BBC3C9A6D3CFF797CA295
:105B8000632A2D9AABA7A68FA670C3CF1AA90E7C45
:105B9000ADCF2934A9477C829975142C063E88A97B
:105BA0003DF8F0BD47D88FCF48814A793F42D30BAB
:105BB0003E4CD3376D49F1DCD5990975B27A2D0287
:105BC0006374E488AEBB18126DF2AFA97E93221DF8
:105BD000292C4BE85963E9D7D62C1D0350A871FC3A
:105BE00093FE9E70A6B43988AABE1A58958B83CCB2
:105BF00025DCFA7B1EF2AD35732724F9742A5EBBCF
:105C00008E5042326A3E77B3E8E78DE7EB349CDD95
:105C1000CCD84888FE7700499EB1D19CF25EF5C38E
:105C20000D1C5E6B2D89E1EB43319AE997541B4FB4
:105C30008D1BD133B8DEFEE25A0C91A733C6BD44AA
:105C4000954182C69CB75EB1EEC04BCEC37F6CA9B6
:105C5000334A5BFC93A9D0509DEB8E88053577D6EF
:105C6000F34BF59755C4D79F20038EE4245D77F45A
:105C70001909E472C3CF09B17EA13D13D8686A0344
:105C800075456FEFE1A90738B852B4A196006A8E46
:105C90008BE47803D5E2DC39170B3E9084B824B24C
:105CA000A9F11D3957B8099AED18776CF089DA27F0
:105CB00057F275A0E391C8A95494B1E7F3528568EF
:105CC0003A59242CE17D51A891CEFBFE2D16E7C058
:105CD000BF72CDCED86026D77F8CBC85362B38A43A
:105CE000A144F34A12BE8EDD65B38EF3CC2098BF7B
:105CF0006E9695E7456BD35006F622404F825927A2
:105D0000EAF0616D8E501D14854F93E39F795132F7
:105D1000E363398D4B8F61DAFB384EF7B555A199A6
:105D2000EBCA969684D4230FEC72BEC695E25DEE64
:105D300042F1BAC5711A857FADAD339100E354527B
:105D400074507D4BD129ECD47DA0E01F208FAD187D
:105D50003F7C721B165D806278050A836CA8753ED5
:105D60009A2A045A80245FE8BFDC050149892CDFA8
:105D7000022ADBCAC16B9706164EC7C61E1E958E39
:105D8000EC8987092D343A0056B5C6558F2B643AF5
:105D9000EB1C6D18B3E4083251AF79ABB5A3D471E5
:105DA000FB486ABC5FB61C5856A58212CC3F020E57
:105DB0005D2203FC86FD3E2E7BD0F353E7A8E92B42
:105DC00017F69917F9B0533F4A9D0B45C3D397F285
:105DD000AE73DDF18E0776C08F8F4C4BCA98029759
:105DE000585306D7D1796143ED608846A465EA0C23
:105DF000C17363E7F5D9309643930E3D180A5D27CA
:105E000062FCD841AFD27408C0AA9571FB5A5AA45B
:105E100067AEFA5E0004E6C9D12EE3A8EAA1C31872
:105E2000A4B20F694A080E1294590DF5EB49A2ABC2
:105E3000579FECA01697009A876ECC27821872A401
:105E4000B3D045540A3B53EF6BB6EAE8083E6E9C6C
:105E50003C06B39C88657FC0B07B4087B68D4D20E3
:105E60000E15607FDC8138D2E58A85AFC1A8EF2DA1
:105E70000BAC92344346E971852A91AFE3863BC669
:105E80009531210B8FA78558579A753B85B8DBA2B2
:105E9000B0B8927707432918126BD5993ADFFAC642
:105EA0000DAC78C3EE87DB9CDAA767CD7E83C88B09
:105EB000D7663C00C54FE9B4DB92BF591983C62BA6
:105EC0006B458C8E5FFCA2598B936EC240D5C5E9A1
:105ED000A1CB8CE1783F6AB57AE783EBAAD29185B2
:105EE0008A744DA232B1766CA21BEE7C0A44652105
:105EF000B59D8164BADF3E0A5481260BD2696CCF0E
:105F00006A90577D3519B3C0B122B175CC5F080CCA
:105F1000032A805E05A177F3B0990926324A955B82
:105F20009A8512483CA8B2DBF1CB498228725EDB2D
:105F3000686B7265FB88EF3F4FD03951231142DE09
:105F40002D61334EED84A5B694D07C96186B4674C3
:105F5000BA8BAD36AB2A98A2FB6F42B1F42D034A3F
:105F6000ECB8874B811AE946D0CDCAA36B099C36A1
:105F7000358C367B8D5E08A8235843149D52235FD1
:105F800013F7CC8175A1D4E749663E2FF20662F77C
:105F90003B18CB836F863F31682F95CF7C655EFAC7
:105FA0006BED5FF67D408E4F6459E044EABF04D448
:105FB000A4F5AF9EBD3EADEC24E98B4263AB6F3FD1
:105FC000EFBECF2771AFBA111982560F9C9A76484F
:105FD0004DABA6B87B47B4BD6A9FDB73C5D4F9B39C
:105FE000FF3DACCF226AE4DEB56CF89BE03251DBBA
:105FF000BEBEED80A3123110FE49A273E61BE0A5E0
:10600000794D522908357E8A2C5AE5165C5A2F2084
:10601000120BF0CABEA30918EA90CB9CFD666F9CD8
:10602000D78E8ED60169A248012FAA669445391EE3
:10603000C326C6F0FE240DEFDA60108B9FB70B98D5
:106040009A9DA84FE131F45E1BBA37B4E136B31B19
:10605000F713549BF04BD2E87A364B51E0710C5F4A
:1060600045638798B5B88D679A745F140C9539BDF0
:10607000A50A71C7E65E3F2A6D38BB9A983DF83E87
:106080003DA29A1301AEDE225FC2AA21135EA5864D
:10609000BB2AA8D7274859AB569C15ACC9CF8B3D16
:1060A0009FAD14680139C3938B35FEAA9D05622B01
:1060B0002AD11D40A61AEE77F06BF69B15393EA744
:1060C000F759965B7533B4DFAAFD872DA7E8FE511B
:1060D000605E0F6AF9FBD64C11FB4709B4E67A54AF
:1060E000F5574D7A5930F7908C957A7ED33D3A32F8
:1060F0005C7BC98BF3EEF4BBBB0B029A1FA6DEC21E
:106100008F558F8632AE6584E3EFAE626EFDD6A109
:10611000E0AD0F8DA4075349D14238A0CCD322E77C
:10612000C41621508976133010BCFA861B2990FBC7
:10613000F0EB4784A67DE0FA8378215AFCE7C2475A
:10614000F3A87A77C14211400D5B1676D10AE12A95
:10615000C46BD7745CE11751CC59E5F29BD61E167F
:1061600084C9B5F89DE8A6B757447F49DFAD7D4D9A
:10617000FE14A7DAB6A71B24A1854ADDF9B1063BB8
:106180009DE6757C92A6ACD837FBBE6A880E33714B
:10619000F2DADCF6D336D139830417717FA78D3656
:1061A0003616152BC28B8D9E3BD18EA1946511287E
:1061B0001C662FE6BC6D71F8066712F74A4D33086E
:1061C000AB4D111B54D747AA7E1A9941F81C945C19
:1061D000C905408D1B259F5B0B79F023582BD1A659
:1061E000E983BB0A23E4E5088DDDD2AE63752D3D5E
:1061F000858BBAEF8E03CB14532EA0E9EF834109B0
:10620000BBA2432156E00AD00EE94D748E454345AA
:10621000913410EC348619B58563FFB8755CD6757A
:1062200077C1E2295C6A14FB3ADC6C279AF418F413
:106230003E227F5A2B61CB9227221B5B26A9D0AF2F
:10624000ADD10E51C7A2AB14EEDB25A575F1B69505
:10625000245599603BE10E15E407C5F425C465009B
:10626000DB5D8FD8D09FC17629A3B2ED5B27D29E8C
:10627000D99A0BCF28DD01420F7073F1C085DE3C47
:10628000F665086F2985910C1106351C81A5481308
:10629000F4270C92902D1498584489703449B7C152
:1062A0000138337046D4CECE38DFEFED1E4DFAD72D
:1062B000651E7B6A832078C998287B010CFB0260ED
:1062C000A652682633298F08494D6D1C19033FB427
:1062D000607413BD134679AB9CFF8F8D1B6D4EFF11
:1062E0006FFC4B2EB089D848E12CB91261A16839F6
:1062F00082359F13201E93D05DAB11D69AFDAC0B57
:1063000069F4AC1E5D7E0D82E59D77D2EE0A9CFE9F
:106310005B238ABC89AF22F87434879DFE346BEB13
:10632000D8F4672D88C35833121FECB1CC45F577EC
:10633000110CEF9166AB9481FFD511F146C7104166
:1063400062144E24C7C8C9C033AE63BE0BD7D92769
:10635000214C013324F3B52F0A9DD99DCCFF45CFA5
:106360000965BEF325C718F2AD113C620BB76C2D61
:1063700018E76003BF35BEBD3C17B8EE4C525BC397
:10638000E476E948862CD3D8A0E85308F03AE7E948
:1063900066610DF374FFCAE2EB8BA69CE6D4BDC820
:1063A0009BB185B5D9330CB78EEACBE2AAFCC32FDB
:1063B00060EAF18D2F1EA6207F7D4366B1845C626A
:1063C0001673D39F3FE20180839F6EDA8BC7E0D3C1
:1063D00068AC266422B0606064BA0AE18F003010B5
:1063E000E32F57038D7E9B79A3055C1AE8B600C5A1
:1063F000EF06E0A073887A34E5836BE00597499A4D
:1064000060BA32DF6C13EF841850C846741547CF5A
:1064100094B760E5205D36BC84F48019D4906DB9E2
:10642000FFC0FFE301BB8187F8541F168F6ED9B5FB
:10643000472F3389C1723055CEC1C08CB43C1C0B80
:10644000506923A3D1DD4927CAC769F2BB851C5611
:1064500007FBBE9DFD61F38B0ECF9C68A8EB6085AA
:106460000B65E77124E0B62BDDD86B7849D81F6245
:1064700096E840ED6027D008EC2ACA0518DF64537F
:10648000FA08A1BA04760DC4CBA30FB380C39CBD98
:10649000CC9AA6F47F3059FB1B00E95E89B6B41C88
:1064A000270BD9C420367D622EAF2F8B5F96C72075
:1064B00007863EFDD00B913D02D624D2840520FEF6
:1064C000DE6C355A0DAF6BC9CC2332BF95099E7770
:1064D000E799A515FE56041D81FFEDE66E3171F8B2
:1064E0007461ECADD3228156075A6429B2EF9DF551
:1064F000A51F56349D7073E02AE2DED5CB14CDDBA8
:1065000059ACC590D7A52E61CBBCDF3E5D719E9581
:1065100009E3B410D26C8DDFDB37C71FD243C87ECE
:10652000206049E01336C7B08B505C8EA934248BB1
:10653000A19BCF0FAFF055E22C97C731BA7F45A092
:106540007F8B3E5EDE6A747758610B6F7E02EA5085
:10655000D937069EDE73FA039DB89A650DEF616D1B
:1065600059F97EADC4334ECA6CF2D27501D58FF5A0
:10657000830A63A28BC15B17987BF41E7BF03708FC
:10658000E8FF3901490CAFFA22049B1AB88CE333B7
:106590004750274774B44CADFCE10695B2F5A48C86
:1065A000D097FE6725739E2CC37A86BBD1599781FD
:1065B00043A9C9674AE467091ECEE9B8D417EE2B90
:1065C00036A98038A5A469B5D6DEE283660A9D5A4D
:1065D000A13485C860EDBEC52118652E1AAD5D7267
:1065E0003446530F5E1FC104BDD094A6511F1585BC
:1065F0006263107ADA96E7D8F39F579FB782457F98
:10660000C15B1733D4111381A0526CAC8201159A6F
:106610007B761BE5D0341AB827A9A32BC479F709D8
:10662000B57E05DF57F30ABE3591513D0EE6EEF714
:106630004767F0A5E5214D216A99421E99BFAC75C7
:10664000EE70618918763D32E173D6F74BEE4EAAB3
:10665000BF3A5E3900887B645DFDA03237C3FA081B
:106660007569447123E697F441D6FC519616E834D7
:106670009C4532F11E4D69E3AD27FFAD671DF43A2D
:10668000479EC70004AB98A5E485A3CC477EA453DE
:1066900059BC5BB5A9F72E810B101B4869C5051BBA
:1066A000AC690890E9F8C0FBA81AF76B623CB50822
:1066B000E11379BC6B4EAC3F2A3441840EE328557C
:1066C00055112916E52C907541D8D4C20E514ED2E1
:1066D0000DF1216B05B9530C55236748B0020B0F20
:1066E00025646A501E4D6B1C25BC3D7193FEA11F95
:1066F0001A416B5644B28250B39DD762C5B2BCDA20
:106700004AA8CD49031BA05F00F3F3EE93C4B9B7C9
:10671000EA8071C02BDDDE94FE34838662237175BE
:106720001278242140DF9D2FB4B82FEE6F78D5BAB0
:106730002E2E38756B7ADB9FCF33A6032D3BC5D049
:106740002DD048931D4BE30DB6756E8984723027AA
:1067500069D7C1F4B8CC9C830B541F87B13A85B775
:10676000291AA979052B7A51F2F845835016EC695C
:1067700091B446413DD8EDF2D95354EAA5AF24CBAC
:106780006291A6D0838997A1BD1A6BA52890BC867B
:10679000596BAA1EE72B42DDB32F28B5A6C25CE2D7
:1067A000FCA4B2356F3C3E2A2C1B1927F21C3494F2
:1067B000E15A15A99629047DF2FF0E5079ED3E08A5
:1067C00043B07DC22502102D63C3BE4DB57CDF7181
:1067D00067AA6448FC0D95C7A0940F27EF5A59B6D5
:1067E0002EB070D1C9D2E9E9AA7BE6984E4313EEE8
:1067F0003FDF82D8AF814F49F2A9CA9267B6AB6535
:1068000099A9714AF14FEA5201B476D87C2732C770
:106810008F03B15DE9616FDA89BA795BDE8770F168
:106820004984BF33A39B31E0006794E0B9910C2306
:106830007AB9CF737ED7E052F2F58030DBA7C86417
:10684000AC4627EB3DBDB5BE1D575E1A2D82F091BB
:10685000DDEDB569CF51FB13222950AF74077C5C85
:10686000261871F3969B69F74CCF69A10D48B58B3B
:106870000831FD2C2AE65896D88E816DE61CAA7543
:10688000EED5E31C04B416803CF33014703F7CD288
:10689000623AA1301B8A47D4C852F16BAF30D6118F
:1068A0003C418C61946B796A5C124F43AD842DE25C
:1068B0001A1F2D6F195DB2E9E5AEF4E92A5061396E
:1068C000D2D44C90060E91CA9B0FA3B64AD0DCFBE3
:1068D000707D2938E6388A083BC1120B12B4C7AA6A
:1068E000B5FC7EE056F6BFBB7EA6AA7B653CC9F729
:1068F000695EBEF9FA194463D069EFAAEC41AB7E38
:10690000D9F1F988BFF875851839430B639D639FEA
:10691000C53040C22A5927096E33821C0C72B73D1C
:106920004CE210FFA8C9D1B7D4DCEC46E6E12EB1A9
:10693000E451365086332C4A02DCF0E4B1BEA93B68
:106940007A27D467C4F6E124677C4BC867E3D7791C
:1069500020597482C8B70D4E5866C23D6DDEB1F441
:10696000AC0680234B1FDEA8A066B97D87184D8A30
:10697000F50CB3A6F45474FB30833B03413A084D45
:10698000169B6C85B77F7725B0515C770A72F25100
:106990002D60BD8F7FB02CB615EED526EA69034574
:1069A000A0F9696F50F5C6BD05DDF548DC0820CCBF
:1069B000875AF7C0328D36A3DEFA8433B93AFF180E
:1069C00073713ACA1C5E83D6E9BF1174AB375FBEE0
:1069D00086B9B1ADDA61E4BEE2573B8173FDFA815D
:1069E000436951F7DFB4673BA55FFF5191044C7ECB
:1069F000BE6F4B01230A701DF3DDC14610DBA7C239
:106A00000D68031720373A64BB1AB89250F72D74FB
:106A1000C1373B8D4A7A7E9AADA0DCF4F953CC8025
:106A2000857CB9B508317A92FF5552265CEF8758BC
:106A300031239105C6486D8C6721105838130B2BF4
:106A4000187CC415DCC5837841B6A4BA26BE871A63
:106A5000D986E0D43D3E98684FECCB57139C36580E
:106A6000B5D8B39A34B69EDB26CADBA9BFA3A5F37B
:106A7000CD0604AAF65FDBF54D1A62B928ECBE0A12
:106A80008EB7DA226123CCA5A38724E1794438B4F8
:106A90008C6827573844DD145382AB2CB1DB16A326
:106AA00072A993FAB95C0323FB8B78411B639BD7D4
:106AB0004FF608F48A3C6F45623ABE8D9A6D12BE5D
:106AC00017C654B59DB94331FCC364EF930B9F5C6B
:106AD000ED373DD37C110945AC55DEDA8ABDA28085
:106AE0007713D1A3C32051832F20A2E11463D6359D
:106AF0001E98F9D929AC0713A874C13E6F27B57346
:106B0000C59E4DB1CCA55A116C19C9CC6BD2F37985
:106B10000BF125A3BAA3EE6DDE6F92E33D4E9D739C
:106B2000E938E06ABC188C9D8758269AC1252B212C
:106B30004D9A72D14ABF0C1877E358ECFA6FFDB743
:106B40001D32A34F41442F0E146EB589B83AB3409D
:106B5000679AC780369B8B774E0DEEB2C4A0DC5986
:106B6000F35AF233C49939614D6CBCAC50D9C09919
:106B70004B89D93F058F6988E5BFE07FF5518926AC
:106B8000583FCAB169FB5962B729BA5D528895F27C
:106B9000BB59898F46F6A5A66FD14FDAEC373782FD
:106BA0007F756384AC8C0A4F123DAAC415B1D3091A
:106BB000B30742D8CEFF9983B4B69A0131263CA9D7
:106BC0005E0F09B3683F8E5E8D1CC7189DED33269E
:106BD00076B1A3700F8ED8C35ABC32B4D7D1F95650
:106BE000026FEB1BFF1ABCB43764C5984C830D5C75
:106BF0004BCD7C43C99C7BBB9C3CA7A5FA4F0CDECC
:106C0000570F9C364A225F684A90F6DBE2DFFF238B
:106C10008917873DC73FFA358759ED9D04A7B00F07
:106C2000B3B9495B692DF031D1C80E36BFB606D075
:106C30003C0679D9480142498349D074458FB21244
:106C4000CB8F14E5E4132675F3134F6277A87164B4
:106C50004BA8650220EDB409CAD51FEC094384B7DF
:106C6000043E7CFB40B9E41DA81DD9AAE1C79310DE
:106C7000C4DF99B1DF374086ACB8AA1D3A7501660A
:106C8000756D1C34C1914A62D2864C3EFB6FA8E8F8
:106C9000EBD61BB9C5FAB5B157CE65E58433C8A4A8
:106CA00011BBB6E92A79D0AE7FE70E6EAB1A6A63E4
:106CB000F3D998EC27BC13EC0BDE1CB5D506B1B1AB
:106CC0001BC4A004DCB2C5DD98A1155BDB6217D93B
:106CD000B5E00E5A4800AFD08CB6423B1282FCC8D9
:106CE000378F2D85A7B03BCDDBC94CFFFE159DDA54
:106CF000E2AADEEB08A921FA517FDD71890E895FD6
:106D0000BFED13D54EF80AC0C97F5E3A522DB38647
:106D100048907F04E2A694779F9815324A22A39662
:106D2000DBBE3AAA2888EBBF7F7FEDCC8C8CC627D0
:106D30006871E2059AC2D76DF9BBD7719D06A4139D
:106D4000557F4BAE3CDC077658270C3EAFF366AB65
:106D5000E28ECBBDE229FF5BD350255AFEB1A3D80A
:106D6000567E285262992130C5906E0A807AB139D8
:106D7000B1B6A5B5CE2E1BC8A8E1C17083B2D0AE06
:106D8000D3A7510AA834E06610B001E5E7D1B53ABF
:106D9000204BFBB41E236B3FC00D6958996B0186D5
:106DA000B2EE0BC7E537C6087C3F985977E5E7D6C2
:106DB00067A09C98A3586C2EEF9960049D78A2C19F
:106DC00057EEAE57F7B2968DFC013FBF2084B2A4B8
:106DD000E3CC8ACF607F6ED79E999EBE106073E72A
:106DE00099DD4B114130A838EAA0872C34718238E4
:106DF000CE046BDB26DEDC161FF28B51693EDA44D3
:106E00004670C1578A352E5B9BE6C5F914CE8DA519
:106E10009D995989D33B2CBD00764E76DA54EAD73A
:106E2000996915F8EF98EE9B501DBB8E290347EC2E
:106E3000BE0151084E2B51376C676124C039F935BA
:106E40008FDAC80C85DEE9C70DD814C38B7C1229F4
:106E50009E23D6286A0EA73B09FA88825F257C48C4
:106E60006B139B80E788870CD08FF921D305AC2466
:106E7000B04451310FB55F5AB61DCE1240354D2B7F
:106E8000531B5A5E113A184CF26D29269E1CC305FD
:106E9000A52084BB7BDE659B5EA00237DB621BF70F
:106EA000AA22E7203FAC2301D0CC5ADA002F96B8B3
:106EB00099F616EABA6824B7BE058ECA11D41D2702
:106EC0003EF3630A9FE76D00DC5FD7908B342F9809
:106ED00045C93A90F7CFF35A6A084FCDA7CC005076
:106EE000BC06496263D372CB76E426D308F9A21BB1
:106EF0008849857ECC3D3E8ECD67889D205DB9EB6F
:106F00000E338FB59E671ED6E75AF47A9938EA8811
:106F1000FE7990359C2A697284EB06405301711BFF
:106F2000B012763809D64B042BEF156C8A79B9FC70
:106F30006F5E1EE364451D8F7119D5D6D88818B3CE
:106F400011A113B69998A8363EFB6D97DBA086E693
:106F5000197282D4868773F3A0B5DDCCC9389EA69A
:106F60000FDCEF901CFBEF0179DF6FEB91F59C36A6
:106F7000E8B9673E474EDF143B032B0F92B8681EFB
:106F800001BBC28EAA98D0E7D2519A1C91FC154140
:106F90008414BEBCD852B881D5B880A292FC036FCD
:106FA0003444519B0FC50AE41C9E532AFB01BA309E
:106FB000BD00FD9CDAC0B3E5FB9C7373DD44E8F4CF
:106FC000CB7F7066C6D6E6ECD30A4C26DF212DBBFC
:106FD000F2DE689E8EBCCC030E176B473AB0F0838E
:106FE0000B6C03EF43752A23FBE92B075EBDFEB351
:106FF000B44E5E8A8BC94D036BEED8DB8C2B8E5E54
:1070000079348CCD477D120075AFFFAAF1230E981D
:10701000ABF22C804D9401446140AA763C853887C0
:10702000149C5B1C7E195BB705FCF38F656E007DBD
:1070300096C3D856DD164353C5E3143E026C36861C
:1070400022DDD13BDEE7AFF9C73F0E2A395B5F187F
:10705000BF10B8CF114731A11A216D82A2ADFF7EBA
:107060002E32A178A78252939A2E7A9A60555A208E
:107070005366C11172FE1ED72D353782A5D2C03E90
:10708000B074A6306909B1D24267311E0F706CEF3F
:107090004B5A155C477C6F825379A3FFCD7FDECEC0
:1070A00063018A1131C3E580EB9E77C71285CEDA82
:1070B0005E9B5C7157565E07DEBDA7DA9B959B5EB3
:1070C0007C049272CAC027C6898389F16A212FD5B0
:1070D0002FDB3561C01608C3BFB6A579E532095963
:1070E0004238D1EA62CA67900762698DB5A925E581
:1070F000C200B4C257B612762A577DB4D2C5913CAD
:10710000B863FB13E6353DABE0A796FE4F2F302169
:107110005EA40BB85B6DABAC40097345C3A007FE22
:10712000C6FC9BDC45F83AF47786FF13D71B3B6718
:1071300084C7FDE1839459F99764E6B078CD1C5774
:10714000A17511846DC055867F7D3552F04088B29F
:107150006B660F3505E36167381C9354001AD247FC
:107160001CD937C51D4CD0620D9C50DA6F50EAA671
:1071700023C93DEFD99D86A32EE64E0DAF34ACF961
:107180002CEC277BE733A39DA9F1400F7F1AB0D0E9
:10719000F5B0289F60B811447B5742A39CBA515E5A
:1071A000AE2EC4D35FAB5BED4908DC6080401FF1BD
:1071B000E1CAEF78A0FF540A83E5940F2747FAF756
:1071C0009CE063C488DB066A485B630C2714C34FEA
:1071D000EE7E2433D080536A21B608B0B4C3DA19E6
:1071E000C2CF0AC1AF4D34847D2FA8819D7E075D3B
:1071F000505BE768CCCEB4AC23474D07E83A57F173
:107200001BAD4A55584B9067A9CAA74EC23ACF50FA
:1072100031A2A3891A8B48957B6E85F3CE954021C8
:10722000202DA4E0A5D3DA885957AFBBF48D7CB6E6
:10723000586D4CBE3C12F0C1FC535797BA342A43E8
:107240008042A24FD538900BBAC80C7880D6ED7C1E
:10725000D171F5CCFD996F5E2FA85041CED4E1924B
:107260003840BA5E7CF247DAECF039D8867946EBE2
:107270004F097571D90029813A6CF24E2A9EC1AB33
:10728000517C3F62655D7E8F5071E0F70C5AEA9346
:10729000AA988610D0E8C84AD89FE5B31258500380
:1072A000518690E053C86E5956DB1D7D4CA2720387
:1072B00092B931B08C9E36FA824BF77A1ADBFB26F4
:1072C00084F19A5767D1A3631D6564E0EE909FC96E
:1072D00055610CADA8DECA3BB3E8E826E689CAD002
:1072E0008D89391856EB283F13976ACCD24680F225
:1072F000F4D1068AA77FC52A4AABDB24E467A188BC
:107300008C9C3CD6C7E6C17B6DE515A9422E8E311B
:10731000CF2661018EAB420C1D9057234FBF3856CC
:10732000B0C13DAE53FF2B76F245FC566C4C724615
:10733000297A2EB310F9A2F88A4C8416C150252060
:107340005DD6A69368408998D9CE59724F4074296A
:107350005FBCCA7A425CDE777C0A413D9E123F8860
:10736000020F820D36B68C9E71D566F39BBE43D953
:107370008FE4BBD602F9B557CC449C6A640E54EF37
:10738000BDF25FE4B5E32459442B617685AE8BA84A
:1073900069CADFD5DC745F89AF8767848464E35E84
:1073A000B5B959E41AC401B5AB2BBAA5FCADEC8450
:1073B000D289A6013EB8F2E1977745E4ECADEC96B0
:1073C000065782958B968ADBF3F4C2D1D206699573
:1073D00041FE94C49441D24548F44F5302967FBF76
:1073E000CE2B3C856377A4C8E1886D56CC986C4859
:1073F000EE83B0DD740F01E0D133C2B18F7E35B3BF
:1074000053E6A6715933DFA4F96FB08705BF6EF05C
:1074100026B530D1F27ED4CC77C9AC15CE274366E1
:1074200096111E577A97C29A212F9EC50280B07B73
:10743000E82ECAB439B55E6B3F04DE21D9B5D92434
:107440005FFE347A0C00DDFCD581C7B5D8B6F68373
:107450005B7402659B010BFC6BD38FAAF81787EA5C
:10746000F54370C723E68CEFD0BC0182DA7F9E9D86
:1074700055DA5F455A061DBB15E6090C5A4E0497AE
:107480002F8B986487334052AE6751097282202453
:10749000C547688253EBBF8AAC80D39E7996DF34B0
:1074A000E14FB391FDBD7C37C5860660C2979ED281
:1074B0002BDA1203C99E360F4EFB97BC56A34B86A0
:1074C000EA856F2B5310631C04D17426371F8D1768
:1074D000A3DBB5A50742962A2CA8D781D63D7F0805
:1074E0002B37700B96D780E6DCBB56D2408B799554
:1074F000F638CAFE34DE15004EE426E9ABD97FE744
:107500005C48008AABECCC264DE98DE17C746CE9DB
:107510003371BF7C8E44E1902A6715C8D61E57751B
:107520005565AB44B6A3D19E329FDD630FDC81C0AD
:1075300068A49DF1AF715618A68046404DDD7B8B47
:10754000482C82588B7D683588F9F50944D9712714
:10755000EDDEF1A610C27ABA3310C963A8403961D2
:107560006D550B88F7CAD769AEC7AF6D9C97528A25
:1075700021428A29B9B7F3A96EDC2FCD23C1EB8450
:107580001091F0C132106276A037C4030D791E0944
:1075900067B12B6680B07EA611D22BF8F0C38A8E1D
:1075A000768B084644426CA7A691FA3F38D35B6EAF
:1075B0006AF810BE6F4636A8AC47D273964D0B8260
:1075C000722CFBD83D1F918D5CB09BB5EDAA2C634E
:1075D000C296EF8B925656ED289C97F4D447260D11
:1075E0001BC6742AF3E0054550F35C7EE66BEF772B
:1075F00082060FFD65CA9C922608CF497A775D976F
:107600000175AC3409285278987B1469B86578C63E
:107610003190CA4370164D3F3FC28A75C7DC1AF5D8
:107620005E382280444951DB76BA4B3024141B7AF1
:1076300078000F7CF97F1EB9942ADEDC7DB676A631
:1076400006026C86DF2549184912D597D8B9DEE9BC
:10765000EFAA816D2B031C081164A35D3C3E812EB3
:10766000481C4559CA0812CF83A1D7D5EE413292A2
:107670007B158DDE9FB31EA39A9525C3974685344F
:10768000799E11C314D4EC476672712D38444D6B4A
:107690004F27E915EDDF03D7DF4A97BE9CBDD19C8C
:1076A000954DBC89DA527C5D27D7646879479DD1B6
:1076B000039AE0F0BFE38CD63243C0ACFFEAE5E3C7
:1076C000923FA80097F02C22D70F13E49C0BA8B888
:1076D000C6FC0734D0E1769B2D6EB02E8A186FACB5
:1076E000EC8267309BD49BFE2E4041952C426878FB
:1076F000F69E1C38EC487C31BC5591F26400566013
:107700000A75FF29BE90C3FE7BD0BB7DA41C441824
:107710005CE7060E9A62EC507B6F087C3FC9FA7BEF
:107720000EF5A4BB6563C1D7D0A2FED3CCE4D3AF22
:10773000A00A9B9AEE330C62E6CD476803722425BB
:107740008ECA201AADBC403D8F2A5EE10408AA9A79
:1077500000C0AC1A01378D1972627B1AAEAE3B3F86
:10776000960C1FE425CBB8C2E2B87DBC179B0497EA
:10777000904A81B3B53D4885E64D7EA7F994B36143
:1077800093E31BC084F09C3C52B76DB65F99345CA8
:10779000E55F124BD450FD7481D5907AC7E5976AA6
:1077A000C45C19F9E2AEC1FAFB977774904D76602C
:1077B000E5EF9763C1C2805F5B0A812477B2D5E9A8
:1077C00054DB2D3FBCC92ADACDBF140B75B280C47F
:1077D0003D6EBC418665CECF47D2F8FF9B575AA07D
:1077E00066B5A25B0D11834A05752C9183E646951B
:1077F000A7D0C7478EB8C8D4491B5DD92D4E36E6F1
:10780000A8EA52E8043884EE9AAD1AD49CBBF40A74
:10781000A062EBE37F63ED531AE3FB9AA35B6F2057
:10782000615B22C76135342C3CEB766CF60DBD39BB
:107830008336D6945C220D2FBAA87002B709E7A947
:10784000FF73BA2D7B5BAC817B6B810103C9A057B1
:10785000BFE0DA486F831B4FC49C941C3FAB753E5E
:1078600058CD5E97B3A8459C0360BAEFD8698E2ABD
:10787000384CC2362826BF59376098CED048F868B1
:107880003DB6B0C543C2256F9044243A7E80D16E88
:1078900045E1D4A8B65615E28C5AE4A719E331C0E5
:1078A00004E19070402854F561BCFCC871782C4EFE
:1078B0009CD468BA505D2D438BE9EA715CA58CAF0E
:1078C00060E787D8374F6FB75E6A5A4DA114189496
:1078D000E56155118251888922D17D7B484A53F94F
:1078E000A8446258486568AD97A0BAE47003EC6399
:1078F0006CE8D7CF0F0396956408A4FE01637D273B
:10790000A5722D61E2B392A16C0D4F573843FB83F2
:10791000DCED386C66C4F56C1B38F256518F4C6246
:107920000DEE838100442113CEC981B3A1CEDF9B2C
:10793000259EC70A80004AC79E777DAAED9DD38306
:1079400093F048849558B3DAB52C42B3AEA5E2F073
:107950004A20FB8B15705411CDA6A7DF763B42DF82
:107960002255E7F01160C0467131BD825C95274712
:1079700044EA849A8AAA3C8ABF7235491B4194B46E
:1079800072A8DA1A90B24FE4B40006E680F8F4B3B5
:10799000B3057A3828F552F88CCD94DB88855119D7
:1079A00095B915D86FCEEC554706DFEA069A9F6960
:1079B000CB2F1DE0C3E59805EC726063D426ABF5D0
:1079C00068A95210459BA729B0F4E9435C5BD51721
:1079D000E0B3BED1BAE5742D669BC787BF4BEEE31B
:1079E0001E3AF5F864B41F1AFFB8025B655903B27A
:1079F00082BEE81830DEF5585F49D74920BE12092B
:107A0000718EFCB64A0ADA07CF214D0A5296EEF47F
:107A100015A5CFD93F8975CAD13F3D5ABFD71D980B
:107A2000914EDDF7F9F6D4A12ECE63F26A39F1D189
:107A3000ABE63D14D3AFBEE5A6F24E4F73138017ED
:107A400028A1CD672BD7FA7F6F7121E9D1F4186E89
:107A5000CCC198FDBBCCFC9AA0560AEA4519C904D2
:107A6000AC68B5889BA97148B85E02D05829A0FFC0
:107A70000EEEAAA1F744C3827493A23756B0202514
:107A8000B642018E1093D41C738BA1C35CE86DCAFF
:107A9000CEEB31C9C78C7F2AEF6814C98F22EF6BF8
:107AA000BF45FED470F3ECA2888FD60FD40B79E6D5
:107AB0001E6BA49ACBB5B9FC6B19A134C619AABD2B
:107AC000400A6C13D39BB66BD5E7D471797D507A9D
:107AD00057897B8C1C787567873F81F26094E0B88A
:107AE0004D46EE7B54D062261134960BCFAA0ACBBA
:107AF000D69DC4E849E2B04DC04C45355DB480B573
:107B0000D5CD5E7C4DA84F290D6048DCD7D889B40F
:107B1000B38600BF6B7322DA0C200BC91E9CB31C0A
:107B2000BFC68F11CEC7580DF0852BA045FE2ED3B2
:107B3000EAD17B67A070506EDAE78CEAC4DCB0DC77
:107B4000D31A6ED7A3439012CD28EDF3B78C8B19BF
:107B5000118E90663A30D48AB69E54C7A89D4F1DA8
:107B6000AFAD6E131E0250BEA0E504007DFB758113
:107B70009DA14B5F3F561F08D6C806C37C88D6D24E
:107B800048E6EF699E50CFF6E2D630F9CC1C77EF8D
:107B9000E478230303ABD40A724E26ABAF9115B041
:107BA0001A006AAE5C229A81BD2D98495445D5B61B
:107BB000C7E8EE8A4E243215ED0246B9590C3CF95D
:107BC0007D45DA1EC07856D021E9F655AE3794D4FB
:107BD000723595D0084A2C1928E52E33D889C5E38B
:107BE000FC314F965E6BA56F38DCAC350F0C2CE882
:107BF000AF671D4808DC96D2DDA828D869AE93AAE5
:107C0000E0FBF462DB4C16BE3B0873CD2E9D2B16B9
:107C1000A0EDB0F5A6B7597AAC5CEE4DA125B96AD6
:107C200036D028373CF9E51BCC5D90D65417081A9E
:107C3000210A5932BBB54307087051CA966235987C
:107C4000EDBEB799C566243AD6FF4D886E3C78D90B
:107C500058239B98F1842E3300803CCEFB1C3F17A9
:107C6000579BD3F0A7EC3D4CF684409864D11DD8C7
:107C7000700CF4D534B5706C7452EF4F5B828DF29A
:107C8000F6923EC4875BF19352988B9138DDC443E2
:107C900059C315513CA9C34420A9336BB1DBF1543E
:107CA00099F7018EF75B7223BC2D815FC8C78CE307
:107CB0004AF3A1A90254CDD7F35C7A6ACB3B539225
:107CC0002A0E78B5A8D48010044EE27D27474DB522
:107CD0009513F85FEDA4EEE7FCC40B5F9E4B1840D4
:107CE000425976FC90E2ADA456AE9239C177E38D4D
:107CF0002D3F7859B24F7C7E32F5308C91719232A3
:107D000011E3DF4AE886A56D8978ACF90BA33DBD88
:107D10009745E09993D1E4130637D939F9F4B1893D
:107D2000FE250ACE406E82E496F1551C32C21D48F3
:107D300024DB4628C0BB3AD382CAB805B1FED805B9
:107D400041771F29A84DEC1283739D93F191A77D74
:107D50000F6D6774A089265925597843EA29249123
:107D6000529CF057E06BABB06EE2F60E04D51E608D
:107D7000F35F4C0126DFC80DABD2D4F844611DD3AC
:107D800063A9E4AF0B47B29FFC7683771F92539BA6
:107D9000460C9E3780BDA35FBD11AAB2D32112D578
:107DA0000E017B642E19DDB3EA080B74F0376E9C6C
:107DB000B758074FDC12B6AF4E8B95065A18A72757
:107DC00020C4BDCE9F375B4ADC6D7A1974B885B785
:107DD0006C66E3F76AFAD36EF365D80C8583F4B367
:107DE0009BF019D2890E87611EF200D1FD71AC1E85
:107DF000B90F40FD20FA29EA7D7B9F0928198CD60E
:107E0000F4DB80D1DD657104B182FE6B262C446AFF
:107E10003C68987A04F433C09221DCE2C232D08705
:107E20009ADD132E3DBCF3B4FB9831B527AA4B2144
:107E300023127BB411A3D7C7CA94C426B5E5B008F2
:107E40006ECAADA97A4CA9A11C550A9D1176E323EF
:107E5000B5F84E2043279CCCFA65F3D3980669C049
:107E600026960E7D9DC0E7BD73D1664A3BFB6F2A07
:107E700090C5C488BF0791A9783FFE7F5C30BD26BE
:107E80009A57BD9C1EE79853B655A02E75ECAA4F85
:107E9000DD90AB720F8AF559AE6E764C4B0B0E131C
:107EA000A6277E881C10E41E69122023CE4CB9152B
:107EB000954DA8EFAF1795B341922C92E8F343BAD2
:107EC000F3EA707296848D84D81D6BFD1211157EB5
:107ED0009F501E5C9053F553546A064D6C2400F875
:107EE000E1ECF1C38D0049F7F45770C87AF35F2EC7
:107EF00028403CD2CE6C561C07573CA4A2AE8CCF77
:107F00008D50F0E5DA5AF9B662EE72DCC23753CC26
:107F1000CB55BF26A115A0D94B3D53F35C5CF7E1CF
:107F200016CCCA9A25F4A1837DBB7CC7872DFE5948
:107F3000F685D5208FD54E0717A8BD645958D30EA6
:107F4000BF48D843F7F7D3F50FDA26B57EB197DCF3
:107F5000094611736FB7CD90AFE1A8128682A3993D
:107F600031A3752F27758029ADCCDABC92D0BE081D
:107F70007659B60D5927711426CB5AD8B32B070B57
:107F8000FD7B266E67645B110E828559706CD5533C
:107F90008C2F7B911D4CAB258D2A95182109E5ADC1
:107FA0005B5823B54AD2E892156DFDB3727528155A
:107FB0006CD368A22BF9975912D612443058AD648D
:107FC000616354A4FE46677A31C860F4D34BD9D3B9
:107FD0002E14C56FB14B53FFA7A520DFC2D01F7869
:107FE00074904BB73268E62E85F18DF81063CF7E22
:107FF0004776A05B69B421B857E8B3B4A4BFDFB13A
:1080000088D88F75AD99DE45D01967E0CA06B96486
:1080100063887DB53C064F2800D39ECF653B77D063
:108020009DE9E4FBD242C5A8A133321656A311F153
:108030006F4543152DD3188314DF95809916649DE1
:108040001164EEAB10FC1450BB4E89A3946A571315
:1080500062EB98C7CD279EEDB192FD325030FF0EF6
:10806000B1D92C97198EA7E38C469DD12DD09E16A1
:108070001A32EED18AFE4BCAC4C2180C9DB6F2C2A7
:10808000803CCDAA889751B356A5BC444F555ACCD5
:10809000CE70D778ED946639A2AB1C37E9A80219E7
:1080A000AC1D9E17FC78D808AD66AD03C419CEBFD1
:1080B00055FE27AA21B7D6D3973B4891D35343FD0A
:1080C00059D45D73AEDCCC488637BEDAA504B2F174
:1080D000DF8269FFE22CBEA3166AE9A6285D62BEB4
:1080E00007027C86DB8CA52E30BCB0D95E0B56E037
:1080F0007E219CC4D7800C17919841DC8BBD0CEE7F
:108100008D0D1733DDDC4B98310BF5F9334D0B41F9
:1081100056EB0140D29CDEC54AF1C906AD8EE9E0BE
:10812000178E22C7A78B698C6C9989D8674D35B299
:10813000852FEA4CAB8B006BD33CEFAEDECCE03747
:108140007E3C00A1B189719EB85D3910243FDF7774
:108150009CE0B808DD182908CF597A2CFA3A119F0B
:108160004A86CAFBDCC330C1E98C840355336A06F6
:1081700078A316653735F5EC89C14198939EC28E78
:10818000BEBDC7E0781C093A85B4088D4CB85DD8EF
:10819000E2C167D0BA9BB8587159DF95880BDAF8FD
:1081A00014C263E309769D2DE1153F746315BEEE9D
:1081B000C568080F7DEB52AA9EB057C7D3E72E01C2
:1081C000B10D3AE6749F83BE623A5F93EDD4D6A0B8
:1081D000342F119A99E1FF0BD269301B9880698D79
:1081E0008FF881D439002B831C67C03D96AE9BED80
:1081F0007F9A8E6AB51C374997B237759C2AC19D04
:108200000D276C77669686FECF22A0A57ABAAD229E
:10821000402D0F9CA60701A9B6A19A8B523EA0B192
:10822000A4BF55B2ACE0E4D87CBF90DE94E6A1CB0D
:10823000E99D3359CFCA4C3963CCBC2205211BF7C9
:10824000EB2103F90A21DD7BA71722A69C781C6786
:10825000318DCF6644AEAFDDCA6468F5D8DDD64453
:108260009EB00D2D0B6A559EA00BE6F3AB0E792246
:1082700007AB17B64663AEF997FAC5256C54051ED1
:10828000A159CF70007FD45F8184971B45C4CFEF85
:10829000A5ACDCFBBEBB4EB742A0057376333F2BCB
:1082A000638E98899740295D0FC38082340781933C
:1082B000A8E291E84C980DA7D9472587A901F60FA8
:1082C000871F5E228D3CA169F95A3FF89008234030
:1082D0005B0F28803A63D62BB20B665A05904EC7C7
:1082E000FCD0817CD472112CDB74AB86F1C9A7AFB2
:1082F000412293954E2F99E02E2D13F0352645906F
:1083000014A5326C10A2346E2AB2BB5709B0A8D79C
:1083100011DAEDB8800F15696EC665397F13BF118C
:10832000C7FBD24477F81D4FC5F19AAF91034C0CAF
:10833000DCE8B2F731A30D7F60FFF38E0885A7CA92
:10834000AB918C15685A3BE6A649969B4B15CA65BE
:10835000CD3ED30949EA0DE377845F1B0350E9ED75
:10836000EE0D96BE9081AC8692A1FAB95F4B29EED4
:108370004D78010C467880C0E1092C4E5D01786390
:1083800047B6BA5C1579FF5D21B20A1E22EFE7FB02
:10839000D05D48B3BFB5528B99331ECCB7728E3DBA
:1083A000068662F4903E2F719BD08C37CE50CCDD88
:1083B000D889FB51307D31CBE04DF5EBE90D79C724
:1083C0004E2C61A2DEE2C469A221E5B1746088A9E5
:1083D0001A4BA6282A8F40DA19B655DA948F0FC0A7
:1083E0006336FA7E087B2E0D55912EAA0775F4B5DB
:1083F000F3D24A64D72B4F711AD58FE70C5CAE01CC
:1084000055D1B55A6A9D47C2049FC9FA036B5BC038
:1084100084E8851700940293F14A1D912248221F97
:108420008D6847CB0A89097DC10B629DC09944B80C
:1084300001AA321616912CAFDBF865071F51382CB4
:10844000013BD646D53403FCEDC761A1F26EFD9F1A
:10845000814BD02B4934FF89E4F84BDC01488E6313
:1084600098AFEA2AB699F9CA7C2587026E5BB7B83D
:10847000FDCE627EF3194FE8811BD0BB7780E758B1
:1084800028AB8243C1DC94289D3F0F411E875CB11D
:10849000B570A8E038219500A35880C749733B6D9B
:1084A000B12B74A2E547ADAB9A2928CD33B7D07371
:1084B000CDADBAC47D80A7F69B55302B20968CB6E7
:1084C000D4DADEC2F8DA959E09588FB3FC32241054
:1084D000E2DD9B2560602F62E4737B00838B1706CF
:1084E000D3CDF63585E8E20CC1E6BB3FBB4B368EFB
:1084F000F2C707DBB14F92F9F67F4DBC40541930FB
:1085000072ED3A4707F364C2235994048F199DF31F
:10851000C9CAA96B9896F1FF32F5AD257391EC7439
:1085200029E33B8BC502881F28DFC333FAFE34A33F
:108530003824A82BE5B8D43CF2A14EEC1069431ABC
:108540005B5136EC5878A14C4A9A2EBF7B2D9897F8
:1085500070610C4BDF5BEADCEE58A2AEF49D8D74CB
:108560002ECBEFBB8C3B51752CD489A6E40B6D61EF
:108570002208FB85C0AE3A774E7A31C26EC94D25CE
:1085800029F0515A27F6392154E8A76563444BFC7A
:10859000F89F9FAD873D2BE745EB234BB4C057F8C1
:1085A0008BC7897DFE33223C4D32CEBA4A4B5800F0
:1085B0009DF89111AC527820068A29F62CA1886486
:1085C000FCA837481EBCEA86967910CAACC5686616
:1085D000D9057A6538AE551B39A42DA897E977558A
:1085E000D2F9E7ED0AA160959A8EDB9D297825D80E
:1085F000A4A64CAD1A34E35EE44349B05197FE0C97
:1086000093D916B98DE7D62FFFD8CDF35F58EB5F1E
:10861000095C666740A6D15A04C3BC25145A6A1F78
:108620000E80321A7F8328E94AA4AAC0537C022D07
:10863000C0B984D929235FC54891C2854700E39A10
:10864000C3ECEF7673B19746A70A14282BB15800F4
:108650009EC835180AAC050DD708B31F3C239913E3
:108660003B3B9436BF5D2DF4CE18AAF9F72AC838E3
:10867000CCF96DE92C23CD84CF65BB3B2FEF8D2C3E
:108680006B97D6EC0DA5FE92CC70FBC7E8D5D397BF
:10869000529299F0768AB2CDC7FE0719124ECCC815
:1086A0003A952DEA5AFBAD98BE96BD22ED5E725604
:1086B0003AA61AD17FE430597C624AD57CDCF9A70E
:1086C000ADEBFB6D9A15B1AB47511544302B5F45AF
:1086D000B87C924ADDB2C93BEFDC6913DD80363AE3
:1086E000EA527745D16D330C41ADA1ED97D0EFFE45
:1086F000661185B80DF1E267F8671D8F61BCDA4736
:108700001598976B232F1AD6CA6DCF8C8EE3BAD0EB
:108710006EF8F16653E723BE0B26386514FB391556
:1087200001CB95D5A399E6D24C03670CFDF2FA492B
:10873000EB6627210EDAD3F8198E42CCBEC9B1D729
:108740006122B908571C1DDB238A7231B6082458F0
:108750000A13122384FB7817EF8D4D4977C4C33475
:10876000E4384F4A0D1A810F68BC500B15EF404A90
:1087700000944B7BEBCB0AD457090C307B5FFF7323
:1087800090ABDBA85F68D7FEECF66018FF11E190B4
:10879000D999B9CAB62040750E4AFE8315020F6CEE
:1087A000B318A85824F25F4169A57EE395D5ABAC18
:1087B00009738653AF15C0D982716FAC8384C885A5
:1087C00002AB7D9B74066B51313A14E4C8CB582F31
:1087D0007F7C33FB0FC56651F810BA9395206B71FF
:1087E000EBCDD2292D8760CAF8CDBD02B8716228C1
:1087F000A4C3E9A10A758AE6498D6ECF6987F62977
:108800003A4E39E6DB73AEA2F8977B4D73FA35101A
:10881000AB6B47074A421D70B1503EB6F5B5A1BFDC
:108820000A6D0DA718647769285BA3369F2932B7B4
:108830007B5E085A0F30BF9037140AAD3519DD1F23
:10884000688B5AAEFF48F8589B55B4BD736D42E72C
:108850009356A59DDA30BE80A08408FC23595B4264
:108860004A68C78AB7B4D8BFD15D274FD06CB42C43
:108870004FBDE625DC69C41079F09A59B2843A38C4
:108880009460645ACC0FBF05B585B5BE81C768FF3B
:108890004C4F751DBC5EBE44B2488D6078E3EF68F6
:1088A000997FBAA5F735E51D200FF183BCAA35B035
:1088B0002591B3F10165DA394A65877C32704C48FD
:1088C000E79E8F4B40D3DEAC2DF5F3F1501E23070E
:1088D0000A80579D80E3367754DACC45A8F7897F24
:1088E0000B8B62FDA172734B362DA95D417F984EB3
:1088F000BFBB7D1B71D1B58AFA27BF6D03204052E3
:1089000023D2E3055FB43527222CA495E6CCF7C02B
:10891000B70D2D72F245091E05B3364DAE5B05B19C
:10892000101537C40EA2B617CEE7BE1B4FF1647107
:10893000055C4706DF1AFAE9AE6613676C26988D68
:10894000FD245096BCC7050BB6D213615508390BF0
:10895000B6C9175E377A73EF3F9732D0321DEBC737
:108960008C70ED4E36193D0F38A40FA46FA2969669
:10897000770CB5D587BDFF99D2920345E9633C5783
:10898000ADCB07A7335EE476F5EF8C109605523B2E
:10899000764140CAF38D5C053A231E030BEADC6A7C
:1089A00057F2A80E9A44D2241778DB9A18C8D93304
:1089B000C569DA3DC97A1B969E9F120CC5A493B374
:1089C000397E54CA4A8F88DEF5476AA56C63003643
:1089D000F2262A15CAD86A7D00EC3EFD73FA9B1D6B
:1089E0005A68FC4B2F463AE34953DB8E4647155BEA
:1089F0000D83C43D8920478D7DEC329F1FFA6B208B
:108A0000118CB90E29137E970FAD6FD5BF9970CF1A
:108A1000B836CE3313FB094E0A35C87F31A92DD99C
:108A200076F8621690AF81E0F0DD30414F160149D3
:108A3000468EC7B92F48DF8BD78FA500DA937E2EDD
:108A400034DB1F71183E417E602420A8E54B267858
:108A5000CD53AE2DF31E019A590ADEC5AEFE97A581
:108A60009B7CCA5E32D7C8734DE40D69DF9B2A6ECA
:108A7000E5EA44C90BC774B97BFF7A4F6A3BFB8AAE
:108A800070D9E2B57F49A59A145FE02EA05A8F7382
:108A90002E68046D8106C0A448E975314800973AF4
:108AA0009BDF5A6DF95F051556BD90452D2B3A9504
:108AB000E671E0A5CF68A173AC8E30C5CC6C533D98
:108AC0006E33D09C3D9B22336A2DEDE51770FBF78A
:108AD000142A109ED6A7EE06125629C14CFB44F06C
:108AE000FECABDE13D9D30914CC838D7FD03361A12
:108AF0008EC6198533A91E5378413B28DE3DABE174
:108B0000374D960FC69C378AC37114DA14C2A0FD84
:108B10008278312EA0667ACA195C6132BBCCE3C27E
:108B2000D4575B4F7208744BA3019C2E172C0DF188
:108B30009D1E438665FBBD8F251F11A3383D42A4B2
:108B4000195E145C3C356F79842368F4870D8E5769
:108B5000017043CAB7BB00925B9DD19A992456C756
:108B6000707EB787BD025981630B3C5548059D8CCB
:108B7000698647908C6E40058FF728B488AE0C4309
:108B8000DCD31F4A280DB850FCBF57079620E137A9
:108B9000F416F1947E35A165B6F740FBF3B54418A1
:108BA0004D509E4B1004818DFF95A737FB40154F0C
:108BB000B6B926DD21D6246AE3E2201D78AF87D737
:108BC000F82CA8E82BE8FD8BA15F05FCCEF03CA2B9
:108BD00012E3CFC5E7C124C1BB09B9EAB8B705A7FD
:108BE00086B5727E39B1008588FE478EFDCCFAB617
:108BF0008F0B7EA504381ECCCEF9357F8EF6096F1B
:108C00007E323C27D4588A501304D609555A7B0C1F
:108C10007B37CC6E021737B85A59C37E0004E8D6AA
:108C2000FB0D7F9C3CDFCB6B1B7818FE21668E8F83
:108C300037792B18866F09004951F3AD5BDAE23AB8
:108C40006F5957331FCB4C220ACBB3F6469EBBE578
:108C50005EA0A48BA6507B0F842F7941FFE18F0883
:108C6000DB96843460F7703F1EC7B28FBF9F0A0245
:108C700010A579B298B136A5EC1C2482C6E18E0904
:108C8000BB5D38C4DC6377AA9BF33A1AD223B41CC9
:108C9000458E577B95F6B11F901A0EBF05012D35F5
:108CA0006A3BB6D7E55E3B8976125B6E0628206389
:108CB000FDC6448637D52802A73994A1BF05EA9B93
:108CC0009C30AB8FFC169E5003A8EED4116F0CEDB8
:108CD0003861D839A7253F6B600AFDA86E87AAC8FE
:108CE000F36F637738AE91F9DD1F3DFA3721258D9B
:108CF0009265B704371967A1E3A571B849ED6B75A3
:108D00004AF82A5A4F69375CEC5C64F13F1DAB9816
:108D100002DE197C97DB53A50F5687F1E65BC4CDC5
:108D200031CE4C7AE55C886B7F3CCE9FB06B77860A
:108D3000431C928783340B9156DC6AA8BBB70F1390
:108D400037D2CC4F2E272B91F1C878E4588CC2D063
:108D5000579F10AA22998F6EE12DC8B90B2093EE70
:108D6000EAD53F6CAF5A4EC868FA93D95CCFEBDFB7
:108D70006E8401B0463216293B5AC923DF40CEEE3D
:108D800065AA2D316AE91811F14106A59F31CD9DE3
:108D90002CA2F2EA706E2DC6D087F3897C2E0FEEDE
:108DA000049B81AE8FCBB3DCD21AE260FD4A71C95D
:108DB000C6DD0DACD89A999422320105BB966DB9E7
:108DC0004FAEE9394BD83E113774F5CB7329665E47
:108DD00052F3059361F97B41703CF07B88BDC6BAC4
:108DE00045AEE260AE2E30D5476BFFEA1CA842EEDE
:108DF00020609CFFEEE2D7B04A1C7C8E691F64C9DC
:108E0000E5815872E9B266056CF0FD2E59A629C7B6
:108E1000804F652332737D66509023DFE597D6D966
:108E2000659F67217B099D86ABABF561E5E786E42D
:108E30005CF033FC3BAE932202125D40BEE6BC5EAA
:108E40007BBD1BEF4B80ED71965094853B19A404BC
:108E500058B9ABB78B88C908A689AF8B2FBCE98AF4
:108E60009FFF5E9DA9F5055751E887AF1307CE51C7
:108E7000B6160982F6D88EEEB16E44A784ABDB57E6
:108E80001DF3586726B24C5E194BAAB171588E8FEC
:108E9000AC153B78C41A1BD7E15DB8A17DBFD99D45
:108EA000E74E392237D9DB556A90834E2D88D6CBD1
:108EB000B6D73A5FFBBAB0A42362D33A80A8CF6199
:108EC000B5C2339254BD6B015AD9A0C13F4CB2EA2E
:108ED00053AE8C1D33A72F70135DA52232DFFCF437
:108EE000F56CEA794C76A1EC25030F3850FE64B29C
:108EF0009084E27D520CD30B491BDD3C6CE28A1B53
:108F00000006DABB9F2E651837FF97B73778D390E6
:108F10003330B8EFEDF2B917E49350CA1835CA0DE3
:108F20009515BFA15F6F8DDE889A7882D7DF4A845E
:108F3000FE2F166F95EBF7C2A6221465F77726A0D1
:108F4000F27817FD5FAE6183D2A133BF5FD85AFBC1
:108F50001D9F5454DBA6D7882F2D6FFE3793DD401D
:108F6000FAE066EAFC6C89988AE6CFE33EBB9E1184
:108F7000DC1DC57F24F7031DAC6C22D7A07653DA25
:108F8000EB8DC13F32E25E3F16AAE378322652896A
:108F9000A55F0BC1B6968D4DD244CA24FB74D80090
:108FA0001C7B8653D1C9E60F5778EF060E2EBA27E1
:108FB000A9AED2C2252B75DD1F8AD4A2B361CA66C1
:108FC0004C24DEBEB50A0503F85E3F67232CC83D7E
:108FD000E4D06AC314A0366406A20CFBE6A84F3B9B
:108FE000ECEF8B78B709645602A6EAD259E9A87269
:108FF0003DD9BAEA1ABCAEADD44CC31DF2BAF67272
:10900000161D1CDFA84A8A3593FCAD9496BDB8BEE8
:1090100093F504EA5002967142445D5DCAEF97CD24
:10902000DFF4B440321B146C42A15C69673E12E667
:109030009FF1B1AA04676716AD1AD4EE9753CB041B
:10904000E78325B1B4AA42195CCDA1E258C35C36CE
:1090500048AF8ADDEF320F643A491D1993D524F6E3
:109060004FED0D2D26C42F86417BE5D2DD58EFB69E
:10907000BD290741ABE0D27D3381FA8783C89CA02C
:1090800092951EB31E45C3FACDBFC0A3EA0299272D
:1090900009CFF653D3966CCC40FFF16AD79C9BE97D
:1090A0009CCD1F06B467F9B51BA7953CC142C566A8
:1090B00005307086D2E7D2C238F0775A617116A4B3
:1090C000009860CF1CDFAF33868CFA265EA09857DD
:1090D000D2CB91B5FD9229B9396F21A5786D15E0F4
:1090E0003BA8DAF0DFFD35BDD9CA97320CF8C8A825
:1090F000EA3193FD0B729CB678DEF5B85ABFA963CE
:10910000C0BB8BD9DD08AE9FF5683D1AE55BB306A1
:10911000387AF1935DAE2BFE7B6C8E2DD1A9407F0A
:109120007CF269974CFF1F7141D94D7346FA6A086A
:1091300032DADDFE0313DD4D1938B94F72E30F0942
:109140000B433A8A8DDB970A58C68EE538899E070D
:1091500038B19DA3E3C8F6802A1FADA6ABB14E8FF0
:10916000A6DEC3E1683F322A5C915D69FE5531732A
:109170007F8B4E29781BD2C66EFE75BF327CE5C54B
:10918000F4EE6767ADF2558304F4C78962533A1F62
:1091900018BF1B09E5C14400CBB3BA0E63CB7925D8
:1091A000DAF12ED9E701B5DF3667B7A286578EC34D
:1091B0009F6B1F2B1D2210AC37CB5D91C605851E02
:1091C0007F182CAB9A0C09FC0ACC9DE8BAE18161AE
:1091D000C57CDE3235C3C85FE5041A0AAED4A5F1FA
:1091E00015A078967C7A5230E004807F9CF5D939BE
:1091F0006F96C9C3BB10CEAB9DA98E48CD63CB265D
:10920000B133495E31A5E170496C84590A1443C8F1
:10921000B1C5C2D46AAFCE3C275FCE9ABCE9AC11CF
:109220007C2E937B25EF658BAFA7D3A12AE42B007F
:10923000301A58D52ED6BB9CB2B3F8C6E209936B50
:10924000A6809CC7A535D0695FB4B8C1EA58BBF207
:109250002FF6E88D6913EEA559735C8D49E977B354
:10926000DBB77DEE610642BCDCF0DC4FA3C4ECA8AA
:10927000A5D09DD76568A15E0D63D4D1DF3F474C73
:10928000E512CBF72FCDF7B9D7255BE41990C0CD08
:1092900082EB40BD2A22FD31AF913E29D3EB1C6603
:1092A000955233081FB6B65F242E970F4C782BB219
:1092B000D124C6CF8A3432C7F71A590CB7395AFFAE
:1092C0000BD6E8239CFA6DDFBA8C30A71FAF1C09C0
:1092D000FA26E040004D9D2A731DC8DD14EF0BB245
:1092E000EEF1C2D4EED8B645DDE3BC6CD167B0B2C6
:1092F000D6E8F00F9070F2954C729E637616A0B689
:1093000056E1F944DAEC845BAF266CDA57F00C4D89
:1093100085AB08CF759AA47A6EDC409957FD089703
:109320001396B23B18256823AF197595B76995F464
:10933000C74AA36E3D581CE2EAA197A43D4C0075B4
:109340002999AA7362DA292BB53274C10E3D4358AC
:109350009B1C19FD867974CE92FDD9A00EEA5A6A3B
:1093600098AA0FFCB10B6D0A78F414D2C445C41648
:109370009A9EA79E6300326839BCCEE62641B6822B
:109380003B14C7B85E8F22882BA2980DF3A8EBB5CB
:109390009D49BD4C15ED4A817113FEA71D0307A918
:1093A000EE33D33C4EF3C5DA62D61D5FA16EBD86A7
:1093B000CAB318E4EC9FD13C8915212E5E031C82B0
:1093C000ED2D7351A8DB14FED71A867B187E2A6711
:1093D000D54B1065DADAE80190715A729AB513E646
:1093E000B169BEE60981902C44B2AE47F5C94D7112
:1093F000B2288C882C2FA71C741879D99EC84338A2
:109400001CB8A9DBCEA139EC37EB4A42837732FF97
:10941000000CAF0304050A08060BFF0209070D0143
:109420000C00FF2025692025692025692D2569006C
:10943000202025633A256900202020205F5F7C00E2
:109440002C00610044697370206F66660D0A005538
:109450005345520046004700424547494E0052419D
:109460004400442E4D59005052474D00555345522B
:109470002020200066202000672020004245474928
:109480004E20202020200052414420202000442E45
:109490004D592020200043202020000D0C205AEDA3
:1094A0004E00000D0C205AE8520000050000000399
:1094B000072061274E0000FFFFFFFF4D0000006600
:1094C00056000000000000051600007E56000083D4
:1094D00056000081560000FF000000FD0A00008DCC
:1094E00056000097560000F55700000000000029C4
:1094F000090000A9560000835600008557000000AF
:10950000000000C9090000B556000083560000C1E4
:10951000560000000000004D080000C35600008304
:10952000560000CC56000002000000AD080000CF3D
:10953000560000D8560000EC56000001000000ED77
:10954000080000EF560000FB560000ED560000003A
:10955000000000550B00000F57000083560000303C
:109560005700000000000039080000325700008357
:10957000560000F7570000FB570000FF570000039C
:10958000580000075800000B5800000F5800006EEC
:10959000560000FFFFFFFF0F000000F40100000471
:1095A0000103010201010411040F0417041601183C
:1095B0000100006C94000074940000789400007C1A
:1095C00094000056940000879400008E940000964A
:1095D00094000067940000081C242C4448586C74C4
:1095E0000502050804080B08040405010504090820
:1095F0000904060807020602040206010604070120
:10960000030803040C080D020C0203020C010C04F5
:109610000D010D080D0408020808070802020704DE
:1096200008010804090209010A080B020A020108DC
:109630000A010A040B0102080204100811021002B8
:109640001108100110041101120212011302130873
:1096500012080F0812041301130414021401150256
:10966000150814081708140415011504170217012A
:1096700019081A0219021602190119041A0116080A
:1096800016041B021B081A0818021A041B011B04EB
:10969000180818040B04202020202020202020203F
:1096A000000000010000004F940000549400005698
:1096B00094000058940000569400005E94000062EC
:0B96C000940000D357000067940000E6
:00000001FF
